:020000040000fa
:080000000014040000000000e0
:020000040000fa
:102800008fb52000007f220000018800000000003a
:102810000c0007006068250001002000110007007f
:10282000000020000000e000020032000000020072
:102830000000000070500200000000000040da00bc
:102840000000fe004440a90060e020000000e0001d
:102850000300320000002000a00188004440a800ce
:102860000000060091018800800078000000eb0065
:1028700015003700e280400032a0b4009101ba0098
:10288000e280400032a0b4009102ba00e280400031
:1028900032a0b4000002eb00472bde00f507b200c7
:1028a000602ce10004003a000059eb008301e900cc
:1028b000fdff3e00040037006128e1000100320006
:1028c0000082eb00040007001101ba000200e000e2
:1028d000e8ff3a00000006003159ba008301e90020
:1028e0000c0032002159ba008301e90008003200cf
:1028f0000400e00003003a00e280400032a0b4008f
:10290000f5ff370011d9ba008301e900faff3a0058
:102910008100e800e180400032a0b4000000060021
:1029200000000000000000000000000000000000a7
:102930000000000000000000000000000000000097
:102940000000000000000000000000000000000087
:102950000000000000000000000000000000000077
:102960000000000000000000000000000000000067
:102970000000000000000000000000000000000057
:102980000000000000000000000000000000000047
:102990000000000000000000000000000000000037
:1029a0000000000000000000000000000000000027
:1029b0000000000000000000000000000000000017
:1029c0000000000000000000000000000000000007
:1029d00000000000000000000000000000000000f7
:1029e00000000000000000000000000000000000e7
:1029f00000000000000000000000000000000000d7
:102a000000000000000000000000000000000000c6
:102a100000000000000000000000000000000000b6
:102a200000000000000000000000000000000000a6
:102a30000000000000000000000000000000000096
:102a40000000000000000000000000000000000086
:102a5000881f780002047800e100070008004000a9
:102a60004f047800000006000000fa00881f78007c
:102a7000000478003fb99700ea8157008000780091
:102a800080522100dd000700800078000000e00097
:102a9000020035000040eb0000f4780001007800ef
:102aa0004f0478000080fa0000000600ec87470021
:102ab000889fbe008a9fbe008c9fbe008e1f78003c
:102ac000f0b79f0081bf9f00820478000004780067
:102ad000010037000804e800184778000e00fb00ea
:102ae0007f0107000000e000faff3a00d0c2b30007
:102af000804f57000500320000c0e900804f5700aa
:102b00000200320000477800010037000804e800a6
:102b10000900e00045003500e18f54004300320019
:102b200040022000808f540040003c000900e0007b
:102b30000e003400f08f54001a003a0000c3b300b6
:102b4000984f100016003a009840900080c7b300dc
:102b500080cf50000300320080c5b30080cf50000a
:102b60000f003a000884e8000e003700a90020009a
:102b700000c3b300984f10000a003a00984090003c
:102b800080c7b30080cf50000400320089002000cd
:102b900080c5b30080cf500002003a000884e800ee
:102ba000090120000805780000c3b30001003700c8
:102bb0000a05e8009a4f1000fdff32008a057800f0
:102bc0006066b8000e00370070a720000042520077
:102bd000c4ef9f006149b9000c00be00eb0907007b
:102be0004fea97000401fb00cf91de008b05e8005f
:102bf000ccb79f00ddb79f000006410081864900e9
:102c00001b00fb003e0107008000780009017800ee
:102c100070a7200041010700000278000000e000da
:102c2000e9ff3a008b0f540006003a000fb89700f6
:102c30000000e00029003200ffb097000108780092
:102c4000260037008a80550020a5200060c07c0047
:102c50000000fb0000805000160033004240a90035
:102c60000f003c004fe997000200fb00cf80de0020
:102c70000000560081805e00800f5600818f5e004c
:102c8000070039006149b900c60907004fb1970034
:102c9000dfb19700820f5000838f5800050032008b
:102ca00020022000b05a88000086eb008086eb00ee
:102cb00005003700d0c2b300804f570002003a0031
:102cc00060061600e0861e008fb997000300e00042
:102cd000030032008b097800010037006066b800fd
:102ce0000c00be004f0778004f06be004f05be0027
:102cf0004f04be00cf00b100000006009001780034
:102d00000200e00002003a000308e9000500370075
:102d10008080eb001304e000020032000308e800aa
:102d20009300fb0001007800000006000200fa009a
:102d3000f0bf9f003fb99700ea8157008f80e900fc
:102d4000e0672100050107000080fa00000006008e
:102d5000800078001106b100030035009101b10038
:102d600001003c000050a100000006000003b1007b
:102d70000b0035009000b100080034008000b10065
:102d8000070035009001b100040034007000b1006c
:102d9000030035009001b10001003c001000050067
:102da0000000050080017800000178000100370074
:102db0000201e8001204e000fdff3a0002003700c3
:102dc0000201e8008100e800114078000049780025
:102dd0000004e000faff3a0003007800000006005b
:102de0008001eb000200370061f079008301e80008
:102df000828f5100fcff3a00000006006200fa00da
:102e0000889fbe008a9fbe000004be0002057800b5
:102e10008300780060f92f000f0040009701070041
:102e200088979f0099979f000000eb00a09f9f004c
:102e30009a4578000b80fb000000ea00cf04de001a
:102e400050c2b30080cf5500020032000904780060
:102e5000010037000904e9000800e0000b0034001d
:102e60001f909700080178008a0078008f919700e2
:102e70000300010090979f000000e00093003200e3
:102e80002f98970000004400a09f9f00090545006f
:102e900050c2b30080cf5500040032000b04e000a4
:102ea000e3ff3a002f989700890037000000eb00fd
:102eb000809f9f00f0979f00e0979f00d0979f0012
:102ec000c0979f00b0979f00c09f9f0009003700e8
:102ed000a0b320000080500000004000e1b22000bc
:102ee000e10078004f98970001007000c09f9f009c
:102ef0000a05e8001a4478008800fb00a0b320000f
:102f000063010700800078000000e000f0ff3a0055
:102f1000a0c2b300804f54000e003a00bf88970053
:102f20000180e900b08f9f0010007800b09f9f00e3
:102f30000000e00005003d000000ea00b09f9f0097
:102f40004f9897000020a000c09f9f000a05e8004e
:102f500010003700b19f9f0003fd2f00f4ff2700f2
:102f6000080037003f989700840f5000040032009b
:102f70006a00b9000000410003004000b09f9f00bc
:102f80000a05e8001a01fb0003004100e90f5000a8
:102f9000f4ff3600e0c2b3009a4f10000400320084
:102fa0000080eb00909f9f008a0478001c0037008f
:102fb0008a04e800a0c2b300994f100007003a004d
:102fc000bf8897000180e900b08f9f001000780053
:102fd000909f9f008a84e800110037000000eb00fa
:102fe000909f9f0003fd2f00f4ff2700080037008b
:102ff0001f989700840f5000040032006a00b90047
:103000000000410003004000909f9f008904e800f9
:103010001901fb0003004100e90f5000f4ff3600e6
:10302000194478008800fb00c0b420001801070094
:103030000000e00002003a00004478000100370080
:103040008904e800a87f9f0080c6b300804f540029
:1030500004003a00994f14000a003a0066405000fc
:1030600006003700c0c6b300804f540005003a0088
:10307000994f140003003a0065404000a07f9f0074
:103080008904e8000905e800cbfb2f008f85450087
:103090001901fb0060f92f000f0040000084e800d8
:1030a0008b0178008000780008007800010107009b
:1030b0000000e00005003a008b007800080078006e
:1030c0003f0207000000e00059ff3d000080eb00d8
:1030d0004f05be004f04be000080fa00000006004d
:1030e0006900e100040035006d00e10003003400d8
:1030f0000002b100010032000000050010000500d0
:10310000800078001104b100030035009101b10086
:1031100001003c000050a000000006008001eb0010
:10312000040037008301e80090cf10000400320053
:103130000000e800828f5100faff3a000000eb0027
:1031400000000600a05a80000000e00001003200ec
:103150000000010060b52000000006001200fa0027
:10316000889fbe008a9fbe008c1f780002047800f2
:10317000a0b79f00b1b79f00830078007880570008
:10318000be0007000000eb00e0b79f00d8b79f002b
:1031900000067800dfb49700194578000a80fb002c
:1031a0000000ea00cf05de000a00fb00ccff0700ac
:1031b0000000e0001a0032006fb097000000e80045
:1031c000e0b79f003fb09700120020008000eb00a6
:1031d000afb197000300010000047800c0ff0700b2
:1031e000000178000000e000f3ff3a006fb09700a4
:1031f000e10f4400070032000000e900e0b79f0043
:103200003fb0970088007800afb19700030001003d
:10321000230037000000e900e0b79f0020003700de
:1032200050c2b300804f5500020032000b047800fa
:10323000190037000b04e900170037006fb0970042
:103240000000e800e0b79f003fb0970012002000a8
:103250008000eb00afb19700030001008000780010
:103260001900fb00808f50000a003200e18f4000ff
:103270007c0032006fb097000000e900e0b79f00cb
:103280003fb097000001eb00afb1970003000100d1
:10329000740037008904e8000804e900e7ff3b00f8
:1032a0005fb0970080804500d1b79f0050c2b30047
:1032b000804f5500030032000a04e000b5ff3a00d9
:1032c00068003700a2c2b3000040eb00914f11002c
:1032d00003003a000100e800d0b79f0002407800e8
:1032e000a0f79f000000eb0080bf9f0003fd2f00b0
:1032f000f4ff27000a0037000fb89700840f500032
:10330000040032006a00b9000000410003004000e0
:1033100080bf9f005fb097000000e800d0b79f001b
:10332000dfb49700194478000801fb000300410056
:10333000e90f5000f0ff36008200780000b4200052
:10334000530007000000e00002003a00004478004b
:10335000020037000900e800d0b79f00b8f79f00cf
:1033600080c6b300804f540005003a00dfb09700dc
:10337000914f14000c003a006640500007003700df
:10338000c0c6b300804f540007003a00dfb097007a
:10339000914f140004003a0065404000b0f79f00d0
:1033a0000100e800d0b79f005fb097009000fb00dd
:1033b00070b42000360007000000e00019003a0059
:1033c0006fb097000000e800e0b79f003fb09700a3
:1033d000120020008000eb00afb197000300010055
:1033e000000478003eff0700000178000000e000c4
:1033f000f3ff3a006fb09700e10f4400070032007e
:103400000000e900e0b79f003fb097008800780017
:10341000afb1970003000100020037000000e9008f
:10342000e0b79f007c8057002f0207000000e000fb
:1034300003003c000c00e0000900320009003700e6
:103440004ff097000004e000010032000c06e80095
:103450005fb097000000e800d0b79f004dff370035
:10346000000678000c0078004f0678004f05be007b
:103470004f04be000080fa00000006000200fa00bf
:10348000f1bf9f00010878000080fa0000000600ec
:10349000040037000204e00001003a0000000500cb
:1034a0000000e80010417800814f5100f9ff3a0018
:1034b00000000600889fbe008a1f78000004780084
:1034c000010278008244780003057800e0c6b3006a
:1034d000804f5100d200320015003c006b4050007c
:1034e000804f5100240032000a003c007040500020
:1034f000804f51000f01320065404000804f510065
:103500007400320050c2b300804f510020013a00d5
:103510001c01370040c6b300804f51001b00320031
:1035200065404000804f510019013a0017003700f4
:1035300030c7b300804f5100fe00320007003c004e
:1035400064405000804f5100620032000040e800ab
:10355000804f51000e013a00e700370050c7b3001a
:10356000804f51005b00320063404000804f5100ab
:1035700007013a00570037009180e900010a7800fe
:10358000780090009171780007013700a8609000e2
:10359000c0c6b30080cf50000a003a009400780003
:1035a00064805000000a78001000be004f89de00e1
:1035b000cf91de000002be00020378008203780093
:1035c0001300370010c7b30080cf50000300320053
:1035d000a0c6b30080cf500006003a0094007800e7
:1035e00068805000000a78003002be002003be0050
:1035f000070037001480e900000a78001000780006
:1036000000027800cfa2de00050378008603780070
:10361000049cbe000694be00a860900080c6b30063
:1036200080cf50000e00320020c6b30080cf500083
:1036300005003a000400fb00cf80de0001017800a5
:10364000820178000a00370040c7b30080cf5000e5
:10365000030032006640400080cf500006003a0070
:1036600004007800cf80de0001017800820178003c
:10367000009cbe000294be003800be002801be00bf
:10368000e00f5000e08f5800e00f5900e08f590024
:1036900003003d0078009000d1c2b3000a0037005b
:1036a000081090000018a30003003200780090007a
:1036b000b1c2b300040037000008a3005300320079
:1036c0007800900001c2b300017578000000e800a6
:1036d0004d003700a8609000c0c6b30080cf5000f6
:1036e00006003a009400780064805000000a7800d8
:1036f0001002be006033b8001300370010c7b300db
:1037000080cf500003003200a0c6b30080cf50002d
:1037100006003a009400780068805000000a7800a3
:103720003002be002003be00070037001480e9000d
:10373000000a7800100078000002780005002000e0
:103740000600200007002000049cbe000694be0076
:10375000a860900080c6b30080cf50000e003200f9
:1037600020c6b30080cf500005003a000480fb0063
:103770000100200002002000030020000a003700a2
:1037800040c7b30080cf50000300320066404000c5
:1037900080cf500006003a000400780001002000ad
:1037a0000200200003002000009cbe000294be0026
:1037b000081090000038a300140032003800be004a
:1037c0002801be00e00f5000e08f5800e00f5900c4
:1037d000e08f59000d00320080c7b30080cf540045
:1037e0000300320080c5b30080cf540007003a00c8
:1037f0007800900001c3b300017578008000e800f4
:1038000009f578000080e8007004980078009000c6
:1038100000004500600498008940780042003700ad
:10382000a8609000c0c6b30080cf500025003200d1
:103830000a003c006440500080cf50002800320055
:1038400000c0e80080cf50001400320068405000f3
:1038500080cf500022003a000a00370040c7b30072
:1038600080cf50001e0032006640400080cf5000e4
:103870001b0032006940500080cf500018003a0011
:10388000060037001480e900000a78001000780074
:10389000485c900008487800450037001480e90033
:1038a000000a78001002780068089000cf80de00df
:1038b0000101780082017800009abe000292be00e9
:1038c0003b0037001480e900000a780010017800fe
:1038d00068089000cf80de000089be003400370009
:1038e0001480e900000a780010007800680c90004d
:1038f000080878002e0037001180e9008008780061
:1039000010007800cf80de0001017800820178008d
:10391000009cbe000294be007800900000004500ac
:103920006004980081c7b300080078008501070093
:103930001f0037001480e900000a780010007800aa
:1039400060049800580990000200e00002003d0069
:1039500005030700090037008000eb00effd0700ba
:10396000800078000000e000030032006800900052
:10397000008050000100370058089000100c98009b
:103980000b003700780090000275780006003700c1
:1039900078009000800045000904e00001003a0032
:1039a00059c2b300894878000000e800700498000c
:1039b0000000eb004f0578004f04be000000060039
:1039c0000400fa00889fbe008a9fbe008c1f78000a
:1039d000000478000106780070089000f80090005c
:1039e00001005000880890000100500098089000e5
:1039f00001005000a808900001005000b808900095
:103a000001005000c808900081055000000222000b
:103a100090bf9f0000032300a0bf9f0008109000ec
:103a20000028a30018003a000b00e0001600340044
:103a30008b04780009057800e28f540002003600fc
:103a40002a002000020037000900e0000b003400cb
:103a500058009000c80190000a017800ee805700dd
:103a600003000100500498000000e00096003200be
:103a70006808900000004500600c98008a8454009b
:103a80004240a900ebff3c00780190000200e000fa
:103a90000b00340058009000c80190008c007800a2
:103aa00003000100500498000000e000860032008e
:103ab00068089000f800900001004000600c980039
:103ac000880c90000900e00015003400090578001a
:103ad000e28f5400020036002a0020000200370066
:103ae0000900e0000b00340058009000c80190006d
:103af0000a017800ec805700030001005004980090
:103b00000000e000700032006808900000004500ee
:103b1000600c98008a8454004240a900ebff3c00ee
:103b2000180990000200e0000b003400e80090004b
:103b300058009000c8019000030001005004980054
:103b40000000e000600032006808900098089000d3
:103b500001004000600c9800a80c90000900e000f3
:103b60001500340009057800e28f54000200360089
:103b70002a002000020037000900e0000b0034009a
:103b800058009000c80190000a017800ec805700ae
:103b900003000100500498000000e0004a003200d9
:103ba0006808900000004500600c98008a8454006a
:103bb0004240a900ebff3c00380990000200e00001
:103bc0000d003400e800900018089000808040004c
:103bd00058009000c80190000300010050049800b4
:103be0000000e0003800320068089000b80890003b
:103bf00001004000600c9800c80c90000900e00033
:103c00001500340009057800e28f540002003600e8
:103c10002a002000020037000900e0000b003400f9
:103c200058009000c80190000a017800ec8057000d
:103c300003000100500498000000e0002200320060
:103c40006808900000004500600c98008a845400c9
:103c50004240a900ebff3c00081090000028a300a0
:103c60001b0032000b00e000190034008b047800c8
:103c700009057800e28f5400020036002a00200077
:103c8000020037000900e0000b00340058009000eb
:103c9000c80190000a017800ee805700030001007f
:103ca000500498000000e00007003200680890000f
:103cb00000004500600c98008a8454004240a9002e
:103cc00003003400eaff37000080eb0001003700fa
:103cd0000000eb004f0678004f05be004f04be0009
:103ce0000080fa0000000600881f780000047800b9
:103cf0000040eb000054980038009000904078009d
:103d000090c6b30080cf50002a00320013003c0060
:103d10007140500080cf50002600320005003c006a
:103d200050c2b30080cf50006400320030c5b300f1
:103d30001b00370030c6b30080cf50001b0032009c
:103d40000040e80080cf50001a0032006940500067
:103d500080cf50006e003a007300370000c7b300f8
:103d600080cf500007003c000040e90080cf5000a9
:103d700010003d000040e90080cf500064003a0090
:103d80000f00370050c7b30080cf50000900320049
:103d90006340400080cf5000060032006540500074
:103da00080cf500043003200590037008000eb0004
:103db0005e00370008007800f20107005f0037005e
:103dc000684890000004e0005b003a00f84890006a
:103dd000c0c6b30080cf5000270032000a003c006c
:103de0006440500080cf50002b00320000c0e8003b
:103df00080cf5000150032006840500080cf500046
:103e000025003a000a00370040c7b30080cf5000b9
:103e1000210032006640400080cf50001e0032007a
:103e20006940500080cf50001b003a000700370067
:103e3000280090000080e90020049800100078001d
:103e4000084c9000084878003b003700280090009c
:103e50000080e900200498001002780048009000db
:103e6000cf80de000101780082017800009abe0058
:103e70000292be0030003700280090000080e90068
:103e8000200498001001780048009000cf80de00e8
:103e90000089be0028003700280090000080e9005b
:103ea000200498001000780048049000080878006a
:103eb00021003700110020001c003700480090004e
:103ec0000000e80040049800180090009801780075
:103ed000120020008000eb00030001008000780049
:103ee00050022000808f50001300320048009000e4
:103ef000e18f4000080032000000e9004004980013
:103f000018009000980178000001eb000300010008
:103f10000000eb00090037000000e90040049800b1
:103f200001007800050037008080eb000800780071
:103f3000ed02070001003700100020004f04780058
:103f4000000006002f03b000889fbe008a9fbe00bd
:103f50008c9fbe008e1f780000077800d0b1200033
:103f6000c0b79f0080c5b30080cf5000080032006a
:103f7000c2b02000c2b79f007740400080cf500001
:103f800003003a0083002000b3b79f000a00370007
:103f900080c7b30080cf500005003200a40020008d
:103fa000b4b79f0080c5b30080cf500002003a0034
:103fb00005012000b5b79f003e04be002e05be00df
:103fc00040c6b30080cf500003003200654040007f
:103fd00080cf50000b003a00e00f5400e08f5c00ef
:103fe000e00f5d00e08f5d0006003d006000b8005e
:103ff0006011b80008045000898458000a0559006f
:104000008b855900bfb39700e88f5300030032003f
:10401000f08f530045003a000200370036002000c0
:104020000100370046002000e00f5400e08f5c00e4
:10403000e00f5d00e08f5d0005003a005e08900033
:1040400081012000a1b79f000000e00008003200bd
:104050003fb197000200e90008006000cfb197006f
:104060006340780090df9f0074012000a4b79f0098
:10407000860278008502e900050033008b05d10037
:104080000a85d3008984d3000884d300f9ff370060
:10409000089fbe000a97be00afb397000700e90073
:1040a00021fc2f008f804000008240003fb197002c
:1040b0008202e90012003700afb397008703e900de
:1040c000a7b79f0000806200cfb0970061527800d0
:1040d0003e00be002e01be00860378008703e90083
:1040e000050033008381d1000281d3008180d30099
:1040f0000080d300f9ff3700009fbe000297be008a
:104100003e00be002e01be00e00f5000e08f5800c0
:10411000e00f5900e08f5900d6003400afb397008c
:104120000700e000e4ff3c00d2003700ae609000e2
:1041300080c6b30080cf50000b00320006003c0068
:104140000104e000080032006640500080cf5000bb
:1041500073003a0004003700c0c6b30080cf50009f
:104160006f003a0031003700080178000800e000d5
:1041700005003a005e08900081012000a1b79f0071
:104180000000e00009003200bfb1970011000900f3
:104190000381d8008000fd004fb297006440780092
:1041a00090df9f0075012000a5b79f00bfb3970067
:1041b000110009000781d80080017800afb0970096
:1041c0000100e90022fc2f000f0141000002410024
:1041d0000c003700bfb29700110009008501d8001c
:1041e00000017800afb397008703e900a7b79f00ed
:1041f0000590b90000805100cfb09700615278005f
:10420000820178000300e000030034002fb1970022
:104210000200e000efff3c0003007800cf80de00ea
:1042200001017800820178003a0037000806be00dc
:10423000e00f5400e08f5c0005003a005e0890003b
:1042400083012000a3b79f000000e00009003200b6
:104250003fb297006121b9000c00be006104070065
:10426000cfb297006540780090df9f007701200073
:10427000a7b79f003fb297006121b9000c00be00b4
:10428000480407000006be00afb297000500e90031
:1042900027fc2f008f8343008083430097b79f0044
:1042a000110037003fb197006114b9000801be004a
:1042b0000c00be004e0407000005be00afb1970021
:1042c0008301e900a3b79f000801be002f04070087
:1042d000000056001fb29700cfb2970065527800d9
:1042e00094b79f000a06be00e00f5600e08f5e0004
:1042f00003003400afb397000700e000e9ff3c0083
:104300004feade00cfa2de000c00be000401780000
:1043100084017800009fbe000297be005500370060
:10432000e00f5400e08f5c00e00f5d00e08f5d0067
:1043300005003a005e08900081012000a1b79f00af
:104340000000e0000d0032003fb19700020278004b
:10435000cfa2de0005037800860378000800be00c7
:104360000a01be00b20407004fb297006440780013
:1043700090df9f0075012000a5b79f003fb1970017
:1043800002027800cfa2de000503780086037800e1
:104390000800be000a01be009e040700009fbe0088
:1043a0000297be00afb197000300e90024fc2f0084
:1043b0000f0242000006420020003700bfb2970003
:1043c00005047800cfc4de00090578008a0578006e
:1043d0000802be000a03be005fa89700efa897007e
:1043e0007fa997008fb1970095040700d0b79f0071
:1043f000e1b79f00f2b79f0083bf9f00afb3970064
:104400008703e900a7b79f000802be000a03be00a9
:10441000110507005faa970000005200cfb2970075
:10442000655678005fb09700efb097007fb19700b6
:104430008fb99700009fbe000297be003e00be00ed
:104440002e01be00d0af9f00e1af9f00f2af9f00f2
:1044500083b79f00e00f5000e08f5800e00f590035
:10446000e08f590003003400afb097000100e00076
:10447000d2ff3c003fb19700e80f510013003a0013
:104480000e1090000038a30010003200afb197006a
:10449000f78f510006003e0024fc2f000f0242005f
:1044a0008300420000c3b300914f100007003200a8
:1044b000afb297008502e900a5b79f0000c3b30023
:1044c00027fc2f008f83430080f37a00afb1970061
:1044d00078811100120f98006e00900024fc2f00cc
:1044e0000f024200830042003dfa07001e099000bf
:1044f0005e089000800f510006003d000200500051
:10450000000f98000e1090000040a10000179800c6
:104510000f0037000000e0000d003d000e1090007d
:1045200074006000f00f500009003a007e0890000f
:10453000fe009000010050008e0890000100500025
:10454000020050004240a90001003400000f980012
:104550004f0778004f06be004f05be004f04be0057
:104560002f03b10000000600800078000100370032
:104570000000e8001004e000fdff3a0001005000d8
:10458000000006002f02b000889fbe008a9fbe0078
:104590008c9fbe008e1f7800800478006000900021
:1045a0000000e00001003c00f0ff27000000e900ef
:1045b000d0049800c90090000c0033000100e8000e
:1045c000c0049800190090009901780012002000a2
:1045d0008000eb000300010000057800b00220001d
:1045e000800f550006003a000b0037000100e8007c
:1045f000c00498002cfd2f000f0646001b0037005a
:10460000d0022000800f5500030032002cfd2f0047
:104610000f0646001600370030fd2f000f04400043
:10462000aad79f00590090000000e900d00498002c
:10463000c90090000a0033000100e800c00498009f
:104640001900900099017800120020008000eb0012
:104650000300010000057800080678000400370018
:104660000100e800c0049800080678000085eb000f
:10467000d8ae2000390090009000fb0008007800c0
:1046800083fb07000800500061ae20006144780001
:104690008805fb0000032000800f550033003a001e
:1046a000590090000000e900d0049800c900900073
:1046b0000c0033000100e800c004980019009000cd
:1046c00099017800120020008000eb000300010037
:1046d0000005780080072000800f550005003a0093
:1046e000070037000100e800c00498000085eb00d7
:1046f0001b00370080052000800f550018003a008d
:104700000804e00002003200f04f54001d003a009f
:10471000590090000000e900d0049800c900900002
:10472000090033000100e800c0049800190090005f
:1047300099017800120020008000eb0003000100c6
:1047400000057800030037000100e800c00498006d
:104750000085eb000047eb000b0120001100370043
:104760000804e000b8003200060037000047eb0004
:104770000804e00004003a00ad002000084778007b
:104780001c0037001ec0b300ad002000ea4f5400eb
:1047900018003200e88f550002003a008b067800be
:1047a000140037006d0120001200370059009000fe
:1047b0000000e900d0049800c9009000090033000f
:1047c0000100e800c00498001900900099017800e9
:1047d000120020008000eb000300010000057800bb
:1047e000030037000100e800c00498000085eb00da
:1047f0001ec0b30000032000800f5500ebff320005
:104800000e04e00018003200005e78001600370049
:104810006f805700800f5600010031000a5e78005b
:10482000590090000000e900d0049800c9009000f1
:10483000090033000100e800c0049800190090004e
:1048400099017800120020008000eb0003000100b5
:1048500000057800030037000100e800c00498005c
:104860000085eb001ec0b300e10f450007003200d9
:104870000d0178008a00780050af200027fa070069
:104880000000e000e2ff3a006600370049009000b7
:104890000000e900c00498000e04e00008003a009f
:1048a00020fd2f000f004000800f56005b003a00f3
:1048b000e10f450059003a008a0078006500370092
:1048c000004eeb0069489000110020000004e00059
:1048d00060003a00390090009040780040c6b30074
:1048e00080cf5000030032006540400080cf500070
:1048f0000a003a000b0178008000eb0020fd2f0039
:104900000f004000650107000203be000002be0068
:1049100010c0b300805498000d0037000b017800e0
:104920008000eb0020fd2f000f004000b5010700c4
:104930000203be000002be0010c0b3008054980005
:10494000b900900000c7b300914f10002c00320056
:10495000f9489000c0c6b30080cf5000220032005a
:104960000a003c006440500080cf50002400320018
:1049700000c0e80080cf50001400320068405000b2
:1049800080cf50001e003a000a00370040c7b30035
:1049900080cf50001a0032006640400080cf5000a7
:1049a000170032006940500080cf500014003a00d8
:1049b00006003700290090000080e900a00498005c
:1049c0001000780004487800120037002900900099
:1049d0000080e900a0049800100078000498be0050
:1049e0000690be000b003700290090000080e9000f
:1049f000a0049800100078000488be00050037006d
:104a0000290090000080e900a004980010007800c0
:104a100004087800110020000e0037008000eb0031
:104a20000c003700490090000000e900c004980025
:104a300019009000990178000001eb008a007800cd
:104a40000300010094ff37001ec0b3008b0020005c
:104a500052ff3700010078004f0778004f06be0074
:104a60004f05be004f04be002f02b100000006003b
:104a700080017800d4c2b3000f0037000300e800c3
:104a8000904f120008003a0093cf100003003e0040
:104a90002340900080cf500012003600e381410097
:104aa000630151000400370093cf10000d00320065
:104ab0000201e90080017800e20f5100efff3e00a3
:104ac0000002eb000400370064c079000402e80033
:104ad000814f500003003200820f5200faff3a006b
:104ae0000000050010000500f0874700889fbe0009
:104af0008a9fbe008c9fbe008e1f78000004780045
:104b0000810678000000eb00c0b79f00f8489000d5
:104b1000c0c6b30080cf500002003a001100200050
:104b2000c1b79f000d00e00023003d00b8009000d9
:104b30000100e80030049800e2c5b3008041eb00ba
:104b400083f79f00904f110003003a000180e800b6
:104b50003004980082f79f00b8049000d0c5b300dd
:104b6000994f100002003200090078000100370060
:104b70000900e800d105200045fa0700d0b79f00e2
:104b80008000eb000000e000bd003200090650008c
:104b9000e20f5600080034000c81e9000900e8002b
:104ba000d10220005df9070011c0b300c1ef9f00e2
:104bb0000000e00002003a008041eb00c3ef9f00dc
:104bc000680090000000e00004003c00f0ff2700b7
:104bd0000d00e00001003a00100020005004980091
:104be000684890000004e0000d003a0028009000a2
:104bf000cfb097000100e000050032000080e9001e
:104c00002004980010007800b0b79f00040037001f
:104c10000080e9002004980010007800f0b79f00a1
:104c20000045eb005e0037000d00e000030034009b
:104c3000090078002af907001e0037000d00e00087
:104c40001e003200cfe997000304e0000c003a0098
:104c5000380090008ff097000104e00004003a0053
:104c60000c017800890078002cf907000b00370050
:104c70000c0178008900780028f907000d00370042
:104c8000380090008ff197000304e00006003a001e
:104c90000c0178008900780075ff07000000e00033
:104ca00006003a006d0037000c017800890078009a
:104cb0006fff07000000e00068003a004fb0970067
:104cc0000000e00009003a00684890000004e0009d
:104cd00032003a00ffb0970089587800f1b79f0082
:104ce00010c0b300005498002c003700c9e79f00a3
:104cf0008905fb000b007800010032001000200045
:104d0000000578001e0020000000e00016003a00b8
:104d10000904e00004003a007c80570012fe0700fe
:104d20000005e800100037000e07e900fc8157007d
:104d300063407f008000fb0048019000e14f40008d
:104d4000070032000200e9004004980018009000bb
:104d5000980178000001eb00030001000200370019
:104d60000200e900400498008e0f5500eeff350068
:104d7000684890000004e00005003a003fb097004a
:104d80000b187800b0b79f0010c0b3000054980013
:104d9000680090000000e900600498002ac0b30099
:104da000580090000000e90050049800480190006d
:104db0000b0033000200e800400498001800900047
:104dc00098017800120020008000eb000300010031
:104dd00080047800e10f400093ff3a0002003700a2
:104de0000200e80040049800480090000000e9003c
:104df000400498000d00e00002003200e24f550030
:104e0000040032000a00fb008080eb001c0032002e
:104e100010003700684890000004e00009003a00e4
:104e2000cfb097000100e00003003200bfb197004f
:104e30008009eb00030037008fe897007fb09700f0
:104e4000014878000d00e00002003d00dfb197004e
:104e5000330498001100200009003700480090003a
:104e60000000e900400498001800900098017800c4
:104e70000001eb008900780003000100ddff37002e
:104e8000010078004f0778004f06be004f05be00b6
:104e90004f04be000f01b100000006000200fa003e
:104ea000889fbe008a9fbe008c1f78008005780016
:104eb00001057800020678000100e00001003a00d8
:104ec0006c8557000b047800010037000804e800e7
:104ed000984478000900fb0081f807000000e0001a
:104ee000faff3a00d0c2b30080cf54000500320070
:104ef00000c0e90080cf54000200320080447800f6
:104f0000010037000804e8000c0178008a007800ee
:104f1000080078003b0007000203be000002be004c
:104f20009a0f540001003a000b0d78009a8f55003b
:104f300005003a00e00f5200e08f5a00e00f5b00de
:104f4000e08f5b0014003a00b0c2b30080cf540081
:104f500006003a00e00f5200e08f5a00e00f5b00bd
:104f6000e08f5b0020003d000b003700d0c2b30093
:104f700080cf54001c003a006000b80002002000fe
:104f8000030028000020e10001a8e10002b0e100d8
:104f900003b8e1000e00360020022000b05a88005d
:104fa0006b40400080cf540004003a006000b8001d
:104fb00002002000030028000d003700f0ff2f0042
:104fc000f1ff2f00f2ff2f00f3ff2700080037004a
:104fd0006000b8006011b8000402500085825800db
:104fe00006035900878359000400be000601be0075
:104ff0004f0678004f05be004f04be000080fa0047
:1050000000000600fc874700889fbe008a9fbe0004
:105010008c9fbe008e1f7800000778008106780004
:105020008204780000047800010037000804e800da
:10503000184678000c00fb0029f807000000e0008b
:10504000faff3a00d0c2b300804f5600050032008c
:1050500000c0e900804f5600020032000046780090
:10506000010037000804e8000900e00005003500f1
:10507000e18f54000300320040022000808f540072
:10508000040034000d00e000b00032008e0e780005
:10509000ae0037000900e0000e003400f08f54002d
:1050a0001a003a0000c3b300984f100016003a00ef
:1050b0009840900080c7b30080cf500003003200ba
:1050c00080c5b30080cf50000f003a000884e8008c
:1050d0000e003700a900200000c3b300984f100055
:1050e0000a003a009840900080c7b30080cf50007b
:1050f000040032008900200080c5b30080cf50003a
:1051000002003a000884e800090120000805780040
:1051100000c3b300010037000a05e8009a4f1000f1
:10512000fdff32008a0578006022b8006033b800c5
:105130002600370010ac200080c0500081ef9f0097
:1051400009027800cfa2de0005037800860378000c
:105150000fb097009fb097002fb19700bfb1970095
:10516000bd010700d0b79f00e1b79f00f2b79f00d5
:1051700083bf9f000fe897000002fb00cfa2de0074
:1051800005037800860378008b05e8000fb09700d0
:105190009fb097002fb19700bfb19700c0af9f009d
:1051a000d1af9f00e2af9f00f3af9f005fb09700c9
:1051b000efb097007fb197008fb9970000024200cf
:1051c00081824a0002034b0083834b0084b79f0017
:1051d00095b79f00a6b79f00b7b79f001b00fb00c5
:1051e000c7f70700800078000901780010ac2000a4
:1051f000caf70700800078000000e000cdff3a0009
:105200008b0f54000a003a000d00e0004f003200fe
:105210008e0e78006022b8006033b80084b79f001b
:1052200095b79f00a6b79f00b7b79f004d00370006
:105230008a805500c0a9200060c07c000000fb00ef
:10524000008050002c0033004240a90020003c00a8
:105250008fea97000500fb00cf80de000101780097
:10526000820178000fb297009fb297002fb397008a
:10527000bfb397000000520081805a0002015b001a
:1052800083815b000020e10001a8e10002b0e100a1
:1052900003b8e1000e00390009027800cfa2de0059
:1052a0000503780086037800da0007004faa97000c
:1052b000dfaa97006fab9700ffab97000400e100f7
:1052c0000588e1000690e1000798e1000a0032003d
:1052d00020022000b05a8800f0ff2f00f1ff2f00bd
:1052e0000001be0080b79f0091b79f00a2b79f004a
:1052f000b3b79f0011003700d0c2b300804f5600f3
:105300000e003a006000b8006011b8000fb29700bc
:105310009fb297002fb39700bfb3970004025000cd
:1053200085825800060359008783590084b79f007f
:1053300095b79f00a6b79f00b7b79f000d00e0008c
:10534000080032008b0e7800060037006000b800bd
:105350006011b80080b79f0091b79f00a2b79f006f
:10536000b3b79f000fb097009fb097002fb1970081
:10537000bfb197004f0778004f06be004f05be0033
:105380004f04be00cf01b10000000600020ab900c0
:10539000001bb9000200b8008100420081004300f8
:1053a000000006006022b800060220000000d000c5
:1053b0008180d2000482d2008582d2000000a00049
:1053c0000202520083825a000300310002024200ae
:1053d00083824a000000a1000603e900f3ff3a00bf
:1053e00000000600efff07000400be0000000600fa
:1053f000839f68000100e00002003d006000100093
:10540000e08018000300e00002003d006001110090
:10541000e0811900e3ff07004f00e00002003b00bd
:1054200060001000e080180000000600881f78006f
:10543000000478005001be004000be00040040009f
:10544000858048000601490087814900009cbe0014
:105450000294be000400e1000588e1000690e1002e
:105460000798e10002003100680044001008e800dd
:105470004f04780000000600f4874700889fbe00b4
:105480008a9fbe008c9fbe008e1f78000205be0062
:105490000004be00d4b79f00e5b79f00f6b79f0099
:1054a00087bf9f000000eb00c0b79f00b0b79f0010
:1054b000a0b79f0090b79f0080b79f000d04200009
:1054c000bfb097004fb09700000140000000e0001f
:1054d0000f003d004f08de0000007100c0b79f00c4
:1054e0009e00070001003d0012002000a1000700ff
:1054f00001003d0012002000a6000700b1000700d7
:10550000b60007000f004000c8ff07002200370068
:105510004f08de0000067100ccb79f008f00070027
:1055200001003d00120020009200070001003d0034
:105530001200200097000700a20007000fb297009a
:105540009fb297002fb39700bfb39700a900070041
:105550000000520081805a0002015b0083815b00e1
:1055600080b79f0091b79f00a2b79f00b3b79f007d
:105570000007eb009f0007000020e10001a8e10008
:1055800002b0e10003b8e100010031001e0020007c
:105590000e005600c0b79f004fb297000400e00015
:1055a0000700350010002000010020006011b80045
:1055b00008047000898470000a0571008b857100f1
:1055c0008d06e900beff3a000400e00003003d0044
:1055d000820007000f00400094ff07004fa89700cb
:1055e0000000e00004003a000fb497009fb4970059
:1055f0002fb59700bfb59700940007004f077800bc
:105600004f06be004f05be004f04be004f01b10063
:1056100000000600881f780018002000881f78000e
:1056200095ff07008f87e9004f047800000006000f
:10563000801feb0090ff07008f87e9000000060045
:10564000889fbe008a9fbe008c1f78006e000700f6
:1056500007003d0073000700e00f5b00e08f5b0078
:1056600007003d00320007000006eb000400370091
:105670003400070002003d002a0007001c00200043
:1056800072000700e3ff07000203be000002be0035
:105690000c00e00001003200220007000400be0000
:1056a0000601be004f0678004f05be004f04be0045
:1056b00000000600889fbe008a9fbe008c1f7800f5
:1056c0005100070005003d0056000700e00f5b0099
:1056d000e08f5b0006003d00040037001900070062
:1056e00003003d006000b8006011b8001000070022
:1056f00056000700ceff07000203be000002be00f6
:105700000c00e00001003200060007000400be00ab
:105710000601be004f0678004f05be004f04be00d4
:10572000000006006000b8006011b80000003700fb
:1057300004025000858258000603590087835900ef
:10574000000006000006eb00e00f5200e08f5a0058
:10575000e00f5b00e08f5b0000000600018040006e
:1057600090b79f000001eb008fb097000100e000b0
:10577000000006000200700090b79f00018040000a
:1057800080b79f000001eb00ffa897000100e00038
:10579000000006000200700080b79f0001804000fa
:1057a0006faa9700cf20de0001007000f0af9f00cd
:1057b00004024200250007004f18de0000027200bc
:1057c00000000600e4af9f000804440089844c00f8
:1057d0000a054d008b854d00000006003fb2970082
:1057e000cfb297005fb39700efb3970000fe2f0092
:1057f000000006003fb09700cfb097005fb1970060
:10580000efb19700000006000205be000004be00d4
:10581000e00f5000e08f5800e00f5900e08f590072
:10582000000006006000b8006011b80008045000d5
:10583000898458000a0559008b8559001c002000f6
:10584000e00f5200e08f5a00000006000800be0082
:105850000a01be0000000600889fbe008a9fbe00ad
:105860008c1f78000205be000004be000006eb009d
:10587000e00f5000e08f5800e00f5900e08f590012
:1058800007003d006000b8006011b8000804500037
:10589000898458000a0559008b8559001c00200096
:1058a000e00f5200e08f5a00e00f5b00e08f5b00da
:1058b00002003d000f0007000c00a2000800be001f
:1058c0000a01be00120007000203be000002be0073
:1058d0000c00e00001003200060007000400be00da
:1058e0000601be004f0678004f05be004f04be0003
:1058f000000006006000b8006011b800040250000b
:10590000858258000603590087835900000006006d
:10591000889fbe008a9fbe008c9fbe000404b80012
:105920000506b8008904460060854e000606b800ea
:105930000a054600e0854e000706b8008b054600c4
:10594000040eb800890446000a854e00e0854d002b
:10595000050eb8000a0546008b854e00060eb800fd
:105960008b0546000416b8000a0546008b854e00dc
:105970000516b8008b054600041eb8008b054600ce
:105980000800be000a01be004f06be004f05be0063
:085990004f04be0000000600f8
:020000040000fa
:020000040001f9
:0457f800bdfa0000f6
:020000040000fa
:020000040001f9
:0457fc007f3e0000ec
:020000040000fa
:10000800e80f0000e80f0000e80f0000e80f00000c
:10001800e80f0000e80f0000e80f0000e80f0000fc
:10002800e80f0000e80f0000e80f0000e80f0000ec
:10003800e80f0000e80f0000e80f0000524b000036
:10004800e80f0000e80f0000e80f0000ae0e000007
:10005800960e0000e80f0000e80f0000e80f00000f
:10006800e80f0000e80f0000e80f0000e80f0000ac
:10007800e80f0000e80f0000e80f0000e80f00009c
:10008800e80f0000e80f0000e80f0000e80f00008c
:10009800e80f0000e80f0000080f0000f00e000055
:1000a800e80f0000e80f0000e80f0000e80f00006c
:1000b800e80f0000e80f0000e80f0000e80f00005c
:1000c800e80f0000e80f0000e80f0000e80f00004c
:1000d800e80f0000e80f0000e80f0000e80f00003c
:1000e800e80f0000e80f0000e80f0000e80f00002c
:1000f800e80f0000e80f0000e80f0000e80f00001c
:10010800e80f0000e80f0000e80f0000e80f00000b
:10011800e80f0000e80f0000e80f0000e80f0000fb
:10012800e80f0000e80f0000e80f0000e80f0000eb
:10013800e80f0000e80f0000e80f0000e80f0000db
:10014800e80f0000e80f0000e80f0000e80f0000cb
:10015800e80f0000e80f0000e80f0000e80f0000bb
:10016800e80f0000e80f0000e80f0000e80f0000ab
:10017800e80f0000e80f0000e80f0000e80f00009b
:10018800e80f0000e80f0000e80f0000e80f00008b
:10019800e80f0000e80f0000e80f0000e80f00007b
:1001a800e80f0000e80f0000e80f0000e80f00006b
:1001b800e80f0000e80f0000e80f0000e80f00005b
:1001c800e80f0000e80f0000e80f0000e80f00004b
:1001d800e80f0000e80f0000e80f0000e80f00003b
:1001e800e80f0000e80f0000e80f0000e80f00002b
:0801f800e80f0000e80f000011
:020000040000fa
:10020800e80f0000e80f0000e80f0000e80f00000a
:10021800e80f0000e80f0000e80f0000e80f0000fa
:10022800e80f0000e80f0000e80f0000e80f0000ea
:10023800e80f0000e80f0000e80f0000524b000034
:10024800e80f0000e80f0000e80f0000ae0e000005
:10025800960e0000e80f0000e80f0000e80f00000d
:10026800e80f0000e80f0000e80f0000e80f0000aa
:10027800e80f0000e80f0000e80f0000e80f00009a
:10028800e80f0000e80f0000e80f0000e80f00008a
:10029800e80f0000e80f0000080f0000f00e000053
:1002a800e80f0000e80f0000e80f0000e80f00006a
:1002b800e80f0000e80f0000e80f0000e80f00005a
:1002c800e80f0000e80f0000e80f0000e80f00004a
:1002d800e80f0000e80f0000e80f0000e80f00003a
:020000040000fa
:020000040000fa
:10599800484500004c500000202d00002064000005
:1059a80069730000706c00006179000020740000c9
:1059b80068690000732000006d6500006e750000c6
:1059c8000d0a00000052000045410000442000007c
:1059d8004d4500004d2000002d200000647500009a
:1059e8006d7000002074000068650000206d0000e4
:1059f800656d00006f72000079200000636f000081
:105a08006e740000656e0000747300000d0a0000db
:105a18000055000053450000442000004d4500009b
:105a28004d2000002d2000006d6500006d6f000006
:105a38007279000020630000757200007265000032
:105a48006e7400006c790000206900006e20000070
:105a580075730000650d00000a0000004552000043
:105a680041530000452000004d4500004d20000036
:105a78002d200000657200006173000065200000a1
:105a880074680000652000006d6500006d6f0000ff
:105a9800727900000d0a000000540000494d000012
:105aa800452000002d20000064690000737000008c
:105ab8006c610000792000006375000072720000bc
:105ac800656e0000742000006461000074650000c9
:105ad800206100006e64000020740000696d000001
:105ae800650d00000a0000005354000041540000f6
:105af80055530000202d0000206700006574000049
:105b08002073000079730000746500006d200000a8
:105b18007374000061740000757300000d0a0000c2
:105b2800005200004553000045540000202d00009d
:105b38002072000065730000657400002074000086
:105b480068650000206300006f6e0000747200003a
:105b58006f6c00006c650000720d00000a00000008
:105b68005341000056450000202d0000207300001e
:105b7800617600006520000070610000726100001d
:105b88006d650000746500007273000020740000e9
:105b98006f200000666c0000617300006820000040
:105ba8006d6500006d6f0000727900000d0a00003d
:105bb8000050000041520000414d0000202d00001f
:105bc80020730000686f00007720000063750000f4
:105bd80072720000656e00007420000070610000a1
:105be800726100006d65000074650000727300004a
:105bf8000d0a000000440000454600004155000021
:105c08004c540000202d0000207200006573000035
:105c1800746f00007265000020700000617200005f
:105c2800616d00006574000065720000732000005b
:105c3800746f000020640000656600006175000054
:105c48006c740000730d00000a000000434100005e
:105c58004d2000004f4e0000202d00002074000051
:105c6800757200006e2000006f6e00002063000057
:105c7800616d00006572000061200000706f000017
:105c880077650000720d00000a0000004341000023
:105c98004d2000004f460000462000002d20000047
:105ca80074750000726e0000206f000066660000c8
:105cb80020630000616d0000657200006120000033
:105cc800706f000077650000720d00000a00000088
:105cd8004c49000047480000542000004f4e000087
:105ce800202d000020740000757200006e20000056
:105cf8006f6e0000206c0000696700006874000087
:105d0800207000006f770000657200000d0a000027
:105d1800004c00004947000048540000204f000094
:105d280046460000202d0000207400007572000017
:105d38006e2000006f660000662000006c6900009d
:105d48006768000074200000706f0000776500002d
:105d5800720d00000a0000004456000052200000a6
:105d68004f4e0000202d00002074000075720000c6
:105d78006e2000006f6e00002044000056520000a4
:105d8800207000006f770000657200000d0a0000a7
:105d98000044000056520000204f00004646000014
:105da800202d000020740000757200006e20000095
:105db8006f66000066200000445600005220000074
:105dc800706f000077650000720d00000a00000087
:105dd8005354000041520000542000004456000073
:105de800527c000052450000432000004f4e000046
:105df800202d000020730000746100007274000000
:105e080020720000656300006f7200006469000082
:105e18006e6700000d0a000000530000544f000098
:105e28005020000044560000527c000052450000fb
:105e3800432000004f460000462000002d200000af
:105e4800737400006f70000020720000656300002a
:105e58006f720000646900006e6700000d0a0000a0
:105e68000054000052490000472000004d4f000038
:105e780044450000204f00004e2000002d20000067
:105e8800656e0000616200006c650000207400000f
:105e9800726900006767000065720000206d0000ed
:105ea8006f640000650d00000a00000054520000f5
:105eb80049470000204d00004f44000045200000e5
:105ec8004f460000462000002d20000064690000b5
:105ed80073610000626c00006520000074720000ad
:105ee8006967000067650000722000006d6f0000a0
:105ef800646500000d0a0000005400004c200000fa
:105f08004d4f000044450000204f00004e20000087
:105f18002d200000656e0000616200006c650000c5
:105f280020740000696d0000652000006c610000ad
:105f380070730000652000006d6f0000646500004c
:105f48000d0a0000005400004c2000004d4f0000d6
:105f580044450000204f000046460000202d000068
:105f68002064000069730000616200006c65000035
:105f780020200000746900006d650000206c00009e
:105f88006170000073650000206d00006f64000000
:105f9800650d00000a000000534500005420000071
:105fa80053540000415200005420000044450000b2
:105fb8004c410000592000002d20000073650000ae
:105fc80074200000737400006172000074200000e7
:105fd800646500006c61000079200000696e0000b3
:105fe8002073000065630000730d00000a000000c4
:105ff8005345000054200000535400004f50000047
:1060080020440000454c000041590000202d0000ac
:10601800207300006574000020730000746f000096
:1060280070200000646500006c61000079200000a9
:10603800696e00002073000065630000730d0000a6
:106048000a000000534500005420000044450000a9
:10605800424f0000554e000043450000202d00002f
:106068002073000065740000206400006562000071
:106078006f7500006e630000652000007469000001
:106088006d650000206900006e2000006d7300003f
:106098000d0a00000053000045540000204800008d
:1060a8004f4c0000442000004f46000046200000ee
:1060b8002d2000007365000074200000686f000048
:1060c8006c640000206f0000666600002074000009
:1060d800696d000065200000696e000020730000f3
:1060e80065630000730d00000a00000053450000be
:1060f80054200000574900004e4400004f5700004c
:10610800202d00002073000065740000207400003a
:106118007269000067670000657200002077000060
:10612800696e0000646f000077200000696e00004f
:106138002073000065630000730d00000a00000072
:106148005345000054200000544c0000204f00002c
:106158004e2000002d200000736500007420000010
:10616800746900006d650000206c0000617000001b
:1061780073650000206f00006e2000007469000045
:106188006d650000206900006e2000007365000046
:10619800637300000d0a000000530000455400001e
:1061a800205400004c2000004f460000462000000c
:1061b8002d20000073650000742000007469000041
:1061c8006d650000206c00006170000073650000c0
:1061d800206f00006666000020740000696d0000f2
:1061e80065200000696e00002073000065630000f0
:1061f800730d00000a000000534500005420000001
:10620800544900004d450000202d00002073000077
:10621800657400002063000075720000726500005c
:106228006e74000020740000696d00006520000095
:106238004d4d00002f440000442f00005959000024
:1062480020480000483a00004d4d00003a53000035
:106258005320000044410000590d00000a000000ce
:106268000d0a0000004d0000454d00004f5200008f
:106278005920000055530000454400002025000027
:106288006c640000206200007974000065730000ef
:106298000d0a000000440000565200002050000083
:1062a8004f5700004552000020200000203a00000f
:1062b800200000004f4e00000d0a0000004f0000b3
:1062c800464600000d0a000000430000414d000052
:1062d800205000004f5700004552000020200000c9
:1062e800203a0000200000004c4900004748000008
:1062f80054200000504f0000574500005220000075
:106308003a20000000520000454300004f520000b0
:10631800444900004e47000020200000203a0000b9
:106328002000000054520000494700004745000083
:10633800522000004d4f0000444500003a20000064
:10634800004500004e410000424c0000454400005a
:106358000d0a0000004400004953000041420000bb
:106368004c450000440d00000a000000544900009c
:106378004d450000204c00004150000053450000ee
:10638800202000003a20000000540000524900007c
:10639800474700004552000053200000202000001d
:1063a800203a000020250000750d00000a000000ba
:1063b80055500000544900004d45000020200000c1
:1063c80020200000202000003a200000256c00005a
:1063d8007520000053450000435300000d0a0000db
:1063e80000540000494d0000452000002020000016
:1063f8002020000020200000203a0000200000009b
:106408005b440000464c0000545d00000020000082
:106418002020000020200000200000004f4e000037
:10642800004f00004646000000540000524900009a
:10643800472000004d4f0000444500002020000088
:1064480020200000202000002025000073200000ec
:106458003a200000257300000d0a000000540000d7
:10646800494d0000452000004c41000050530000f9
:10647800452000004d4f0000444500002025000045
:10648800732000003a200000257300000d0a000068
:106498000053000054410000525400002044000002
:1064a800454c000041590000202000002020000039
:1064b80020250000732000003a200000256c000011
:1064c8007520000053450000430d00000a0000003d
:1064d800535400004f50000020440000454c000079
:1064e800415900002020000020200000202000004a
:1064f80025730000203a0000202500006c7500007c
:1065080020530000454300000d0a0000005400001d
:10651800524900004720000044450000424f000057
:10652800554e0000434500002020000020250000b3
:10653800732000003a200000256c00007520000040
:106548004d5300000d0a000000540000524900009d
:1065580047200000484f00004c440000204f000036
:10656800464600002020000020250000732000007f
:106578003a200000256c00007520000053450000fb
:10658800430d00000a000000545200004947000073
:1065980020570000494e0000444f000057200000db
:1065a800202000002020000025730000203a000071
:1065b800202500006c7500002053000045430000b2
:1065c8000d0a000000540000494d0000452000005d
:1065d8004c41000050530000452000004f4e000081
:1065e8002020000020250000732000003a20000031
:1065f800256c00007520000053450000430d000085
:106608000a000000544900004d450000204c0000dd
:106618004150000053450000204f0000464600004e
:106628002020000025730000203a000020250000eb
:106638006c75000020530000454300000d0a00005f
:1066480000430000414d0000455200004120000079
:10665800504f000057450000522000004f4e0000e8
:106668000d0a000000430000414d000045520000a3
:1066780041200000504f0000574500005220000004
:106688004f460000460d00000a0000004c4900007b
:1066980047480000542000004f4e00000d0a00003b
:1066a800004c00004947000048540000204f0000fb
:1066b800464600000d0a0000004400005652000043
:1066c800205000004f57000045520000204f0000a6
:1066d8004e0d00000a000000445600005220000041
:1066e800504f000057450000522000004f46000060
:1066f800460d00000a00000052450000434f00000c
:1067080052440000204f00004e0d00000a00000017
:1067180052450000434f000052440000204f000043
:10672800464600000d0a00000054000052490000cf
:10673800472000004d4f000044450000204f000056
:106748004e0d00000a00000045520000523a0000b9
:10675800204400005652000020530000544100001d
:106768005254000020540000415300004b20000008
:106778004e4f000054200000434f00004d500000d1
:106788004c450000544500000d0a0000005400006c
:1067980052490000472000004d4f000044450000ca
:1067a800204f0000464600000d0a0000005400007b
:1067b8004c2000004d4f000044450000204f0000d1
:1067c8004e0d00000a00000045520000523a000039
:1067d80020450000525200004f52000020450000a2
:1067e8004e410000424c0000494e00004720000086
:1067f800544c0000204d00004f440000450d00009f
:106808000a000000544c0000204d00004f440000d6
:10681800452000004f460000460d00000a00000019
:1068280045520000523a0000204500005252000034
:106838004f5200002044000049530000414200002c
:106848004c4900004e470000205400004c20000036
:106858004d4f0000444500000d0a000000540000a0
:1068680045530000543100000d0a00000054000098
:1068780045530000543200000d0a00000054000087
:1068880045530000543300000d0a00000054000076
:1068980045530000543400000d0a0000004d00006c
:1068a800454f0000570d00000a0000002564000055
:1068b8002f250000642f000025640000202500001b
:1068c800643a0000256400003a25000064200000b6
:1068d8002564000000450000525200003a200000e4
:1068e8004241000044200000464f0000524d000085
:1068f800415400000d0a00000055000053410000fb
:10690800474500003a2000004d4d00002f4400008c
:10691800442f00005959000020480000483a000060
:106928004d4d00003a530000532000004441000040
:1069380059200000280000004441000059200000b0
:106948003d200000312d00003e530000756e000010
:106958002c200000322d00003e4d00006f6e00001c
:106968002c2000002e2e00002e2000002c200000dd
:10697800372d00003e53000061740000290d00000f
:106988000a00000045520000523a0000204d000065
:106998004f4e000054480000204f0000555400009e
:1069a800204f000046200000524100004e470000e2
:1069b8004520000028310000202d00002031000073
:1069c800322900000d0a0000004500005252000064
:1069d8003a20000044410000592000004f550000b3
:1069e800542000004f46000020520000414e000095
:1069f8004745000020280000312000002d2000001d
:106a080033310000290d00000a0000004552000043
:106a1800523a000020590000454100005220000071
:106a28004f550000542000004f460000205200003f
:106a3800414e00004745000020200000283100009a
:106a4800312000002d20000039390000290d0000f8
:106a58000a00000045520000523a00002048000099
:106a68004f55000052530000204f000055540000bd
:106a7800204f000046200000524100004e47000011
:106a88004520000020280000312000002d200000b3
:106a980032340000290d00000a00000045520000b1
:106aa800523a0000204d0000494e000055540000a5
:106ab80045530000204f000055540000204f0000af
:106ac80046200000524100004e47000045200000cb
:106ad80020280000302000002d200000353900005b
:106ae800290d00000a00000045520000523a00003b
:106af80020530000454300004f4e0000445300005f
:106b0800204f000055540000204f00004620000090
:106b1800524100004e470000452000002028000098
:106b2800302000002d20000035390000290d00001c
:106b38000a00000045520000523a000020440000bc
:106b480041590000204f000055540000204f00001c
:106b580046200000524100004e470000452000003a
:106b680020280000312000002d20000037290000d7
:106b78000d0a000000540000494d000045200000a7
:106b88005345000054200000544f00003a200000f4
:106b98000000000053450000540000004845000074
:106ba8004c5000007c3f00000052000045410000ae
:106bb800442000004d4500004d00000055530000e2
:106bc80045440000204d0000454d000000450000f0
:106bd8005241000053450000204d0000454d000083
:106be80000540000494d00004500000053540000c7
:106bf80041540000555300007c53000054410000ec
:106c080054000000524500005345000054000000a5
:106c1800534100005645000000500000415200005a
:106c2800414d000000440000454600004155000069
:106c38004c54000000430000414d0000204f00006c
:106c48004e000000434100004d2000004f46000068
:106c5800460000004c49000047480000542000004e
:106c68004f4e0000004c0000494700004854000007
:106c7800204f000046460000004400005652000025
:106c8800204f00004e000000445600005220000033
:106c98004f460000460000005354000041520000d7
:106ca8005420000044560000527c00005245000069
:106cb800432000004f4e000000530000544f0000d6
:106cc8005020000044560000527c0000524500004d
:106cd800432000004f4600004600000054520000c8
:106ce80049470000204d00004f44000045200000a7
:106cf8004f4e000000540000524900004720000099
:106d08004d4f000044450000204f0000464600005b
:106d1800005400004c2000004d4f00004445000086
:106d2800204f00004e000000544c0000204d000091
:106d38004f440000452000004f4600004600000078
:106d48005445000053540000317c000054310000c9
:106d58000054000045530000543200007c540000e9
:106d6800320000005445000053540000337c0000fa
:106d78005433000000540000455300005434000010
:106d88007c54000034000000484500004c4c0000d2
:106d98004f2000004b4900005454000059000000e7
:106da80000000000ceb5000000020000d2b50000cf
:106db80010020000d9b5000046030000e2b500004b
:106dc800b4030000ebb5000032040000f5b5000084
:106dd8003e040000fab500005804000006b60000a2
:106de800560500000cb600006205000011b6000050
:106df800a605000017b60000b00700001fb6000087
:106e0800ec07000026b60000020800002eb60000bd
:106e18001808000037b600002e08000041b6000030
:106e28004408000048b600005a08000050b60000a8
:106e38007008000061b600008608000072b6000005
:106e48009c0800007fb60000c40800008db6000052
:106e5800ec08000098b6000014090000a4b6000071
:106e68003c090000adb600004e090000b6b60000af
:106e78005e090000bfb600006e090000c8b6000039
:106e88007e090000d4b60000000000005354000042
:106e98004152000054200000444500004c410000cd
:106ea80059000000535400004f50000020440000d7
:106eb800454c0000415900000044000045420000d4
:106ec8004f5500004e43000045000000484f0000a9
:106ed8004c440000204f00004646000000570000c8
:106ee800494e0000444f000057000000544c000079
:106ef800204f00004e000000544c0000204f0000be
:106f080046460000000000004ab700008e09000055
:106f180056b70000a609000061b70000be090000ce
:106f28006ab70000d609000073b70000ee09000038
:106f38007ab70000060a000080b700001e0a0000a9
:106f4800f5b50000360a0000d4b6000000000000c5
:106f580073740000617200007454000061730000d3
:106f68006b5300007461000074650000203d000050
:106f78002000000054410000534b00005f4900000e
:106f88004e49000054000000494e000049540000da
:106f9800494100004c5f000057410000495400007f
:106fa80000440000565200005f5000004f57000098
:106fb8004552000000430000414d00005f500000b2
:106fc8004f570000455200000052000045430000a2
:106fd8005f5700004149000054000000524500007e
:106fe800434f0000524400005f4f00004e00000075
:106ff8004c49000047480000545300005f5000000f
:107008004f57000045520000005400004153000053
:107018004b5f0000434f00004d5000004c450000fe
:107028005445000044000000554e00004b4e00003f
:107038004f5700004e0000000d0a00000d0a000026
:10704800007400007269000067570000696e000054
:10705800646f000077540000696d000065720000dd
:10706800203d0000202500006c7500002053000022
:1070780045430000530d00000a0000007472000030
:1070880069670000576900006e6400006f770000b0
:107098004d6f000064650000203d00002054000092
:1070a80052550000450d00000a00000074720000ef
:1070b80069670000576900006e6400006f77000080
:1070c8004d6f000064650000203d00002046000070
:1070d800414c0000534500000d0a000000740000f8
:1070e8007269000067570000696e0000646f000055
:1070f8007741000063740000697600006520000095
:107108003d20000054520000554500000d0a0000c3
:10711800007400007269000067570000696e000083
:10712800646f000077410000637400006976000016
:10713800652000003d200000464100004c5300003f
:10714800450d00000a0000000d0a00000074000050
:10715800696d0000654c00006170000073650000f7
:10716800546900006d650000722000003d20000099
:10717800256c0000752000005345000043530000b3
:107188000d0a000000740000696d0000654c0000e5
:1071980061700000736500004d6f000064650000b9
:1071a800203d00002054000052550000450d00000d
:1071b8000a000000746900006d6500004c61000061
:1071c80070730000654d00006f64000065200000ca
:1071d8003d200000464100004c530000450d0000d2
:1071e8000a000000746900006d6500004c61000031
:1071f800707300006553000074610000746500003e
:10720800203d00002054000052550000450d0000ac
:107218000a000000746900006d6500004c61000000
:10722800707300006553000074610000746500000d
:10723800203d000020460000414c0000534500005e
:107248000d0a0000004700004f54000020540000c1
:107258005249000047470000455200002025000021
:10726800752000004154000020250000730d000027
:107278000a00000052450000434f0000524400003d
:10728800204f00004e28000025750000292000002e
:107298004154000020250000730d00000a00000082
:1072a80052450000434f000052440000204f0000a8
:1072b80046460000282500007529000020410000ee
:1072c80054200000257300000d0a00000000000093
:1072d800313000003a330000393a00003332000000
:1072e80000530000657000002031000032200000cb
:1072f8003230000031310000000d00000a4100006a
:10730800555400004f4e00004f4d00004f550000ef
:107318005320000054490000535300005545000015
:1073280020530000414d0000504c00004552000021
:1073380020250000732c000020250000730d00009c
:107348000a000000244e0000616d0000653a00004c
:1073580020730000657000005f310000325f00009c
:1073680032300000313100002024000000430000ca
:1073780056530000207400006167000020220000be
:1073880025730000220d00000a0d00000a0000000d
:1073980046610000696c000065640000207400000c
:1073a8006f20000072650000616400002063000027
:1073b8006f6e000066690000672c000020750000f1
:1073c800736900006e6700002064000065660000b5
:1073d800617500006c740000206300006f6e00008f
:1073e80066690000670d00000a000000200900001f
:1073f80000450000525200002025000030340000f3
:10740800640d00000a00000052440000590d0000fd
:107418000a000000537500006e200000004d0000b7
:107428006f6e000020000000547500006520000009
:107438000057000065640000200000005468000048
:10744800752000000046000072690000200000005e
:107458005361000074200000003f00003f3f00001f
:10746800200000004a6100006e2000000046000075
:1074780065620000200000004d61000072200000dd
:107488000041000070720000200000004d61000003
:1074980079200000004a0000756e000020000000fe
:1074a8004a7500006c20000000410000756700006c
:1074b800200000005365000070200000004f00000d
:1074c80063740000200000004e6f0000762000006a
:1074d80000440000656300002000000025640000ef
:1074e8002025000030320000643a000025300000fa
:1074f800326400003a2500003032000064200000a9
:107508002564000000250000642f000025640000a9
:107518002f250000642000002530000032640000a0
:107528003a25000030320000643a0000253000009f
:107538003264000000000000455200004153000082
:10754800494e0000472000004e5600004d00000044
:107558002e0000000d0a00004552000041530000b3
:1075680045200000434f00004d5000004c450000ee
:10757800544500000d0a000000000000200900002a
:1075880000200000003000003132000033340000d9
:0c759800353600003738000039000000d4
:020000040000fa
:100400000200fa00000f78005200200081782b00d3
:100410001e007800062a07000080fa00000006008f
:100420000200fa00000f7800c1cc2a001000200062
:100430007e0507000080eb00041d070071ce2a0036
:1004400010002000790507000080eb00ff1c07006a
:10045000d1d02a0010002000740507000080eb00b6
:10046000fa1c070021d32a00100020006f050700a6
:100470000080eb00f51c070011d52a0010002000b9
:100480006a0507000080eb00f01c070081d72a00f6
:1004900010002000650507000080eb00eb1c070042
:1004a00051d92a0010002000600507000080eb00f1
:1004b000e61c070041db2a00100020005b05070056
:1004c0000080eb00e11c0700d1dd2a0010002000b5
:1004d000560507000080eb00dc1c0700f1df2a0056
:1004e00010002000510507000080eb00d71c07001a
:1004f000a1e22a00100020004c0507000080eb005c
:10050000d21c0700a1e42a001000200047050700c4
:100510000080eb00cd1c0700c1e62a00100020007f
:10052000420507000080eb00c81c0700d1e82a0044
:10053000100020003d0507000080eb00c31c0700f1
:1005400001eb2a0010002000380507000080eb00b6
:10055000be1c0700d1ec2a00100020003305070064
:100560000080eb00b91c0700c1ee2a00100020003b
:100570002e0507000080eb00b41c070011f12a00d3
:1005800010002000290507000080eb00af1c0700c9
:1005900051f32a0010002000240507000080eb0022
:1005a000aa1c0700a1f52a00100020001f05070063
:1005b0000080eb00a51c070011f82a0010002000a5
:1005c0001a0507000080eb00a01c070071fa2a0042
:1005d00010002000150507000080eb009b1c0700a1
:1005e00001fd2a0010002000100507000080eb002c
:1005f000961c0700c1ff2a00100020000b05070011
:100600000080eb00911c070061022b00100020000d
:10061000060507000080eb008c1c0700f1042b008e
:1006200010002000010507000080eb00871c070078
:10063000a1072b0010002000fc0407000080eb0045
:10064000821c0700410a2b0010002000f70407005d
:100650000080eb007d1c0700110d2b001000200016
:10066000f20407000080eb00781c070001102b004b
:1006700010002000ed0407000080eb00731c070051
:100680000000eb000080fa00000006000a00fa00fb
:10069000400798000000eb00200798006000b800b9
:1006a000008fbe0027003700030120008291200048
:1006b0001e00be00f92707000001200001002000f5
:1006c0001e0f40005e9748000000eb0030079800c6
:1006d00017003700be00900080912000008040008d
:1006e000104078000004e00005003d0010002000ec
:1006f0002007980000012000300798000c00370008
:10070000be009000809120000080400010407800e2
:1007100080407800100020008c0407000000e000fa
:10072000030032003e0090000000e800300798000f
:100730003e009000ef0f5000e6ff34000080eb0019
:10074000421c07002e0090000000e000d6ff32009f
:1007500041132b0010002000b40407000000eb0040
:100760000080fa00000006000e00fa006007980002
:100770000000eb00400798006000b80020079800d8
:10078000310798006000b800008fbe0025003700d8
:1007900003012000829120002e009000be009000f6
:1007a000be2707002e009000be00900070004000a1
:1007b000e080480020079800310798000000eb0017
:1007c0005007980012003700de0090008091200052
:1007d00000804000104078000004e00005003d006b
:1007e00010002000400798000001200050079800ea
:1007f0000700370010002000010020001e0f4000fd
:100800005e9748005e0090000000e80050079800e6
:100810005e009000ef0f5000ebff34000080eb0013
:100820000a1c07004e0090000000e000d8ff3200d4
:100830001e00be00809fbe0070132b00801f78003a
:100840008091200088080700e687570081912000ea
:1008500010002000750407000000eb000080fa0083
:10086000000006000200fa00000f78006827070069
:100870000000eb000080fa00000006000200fa0011
:10088000000f78008091200048210700819120000e
:10089000100020006504070041132b001000200009
:1008a000620407000000eb000080fa000000060070
:1008b0000800fa0030079800f3220700200798008c
:1008c000eb220700008fbe001e00be004206200083
:1008d00003002000b3120700008fbe00f1142b00ac
:1008e000100020005104070030002000761f070090
:1008f0000000e00004003200e1152b001000200091
:100900004a0407000300370031162b0010002000b6
:100910004604070091162b00100020004304070036
:1009200010002000681f07000000e00004003200f3
:10093000e1152b00100020003c04070003003700e5
:1009400031162b00100020003804070081172b00ff
:100950001000200035040700200020005a1f070067
:100960000000e00004003200e1152b001000200020
:100970002e0407000300370031162b001000200062
:100980002a04070071182b0010002000270407001c
:100990000000eb004c1f07000000e00004003200e4
:1009a000e1152b0010002000200407000300370091
:1009b00031162b00100020001c04070061192b00c9
:1009c0001000200019040700991c07000000e00037
:1009d00004003200511a2b001000200013040700fd
:1009e00003003700f11a2b00100020000f0407004d
:1009f000a11b2b00100020000c040700ac1c0700fa
:100a00000000e00004003200511a2b00100020000a
:100a10000604070003003700f11a2b001000200025
:100a2000020407002e009000801f7800901c2b000d
:100a3000801f7800809120000b080700e487570092
:100a40008191200010002000f80307001e00be0066
:100a5000809fbe00c01d2b00801f78008091200069
:100a600001080700e6875700819120001000200050
:100a7000ee030700511f2b0010002000eb030700be
:100a800080912000c92007008191200010002000e3
:100a9000e603070041132b0010002000e3030700ca
:100aa0000000eb000080fa00000006000200fa00df
:100ab000000f78000000fe000000eb000080fa004c
:100ac000000006000200fa00000f78000000eb00b2
:100ad000c04a8800561c0700d04a8800741c0700d2
:100ae000e04a8800c1220700f04a8800014b8800d4
:100af000ca220700104b8800214b8800bc1b07004e
:100b0000304b8800414b8800911b0700504b8800f8
:100b1000614b8800931c0700704b8800814b880054
:100b2000e41b0700904b8800a14b8800121c0700b3
:100b3000b04b8800c14b880080952000c823070077
:100b40000000eb000080fa00000006000c00fa0034
:100b500050079800361c0700400798004e00900090
:100b6000e10f500003003a0040202b0010079800ce
:100b700002003700b0202b00100798004e009000b4
:100b80000000e0000300320020212b00000f78005d
:100b90000200370050212b00000f78001e00780063
:100ba000801f78009e009000811f780090212b000c
:100bb000801f780080912000ab070700e687570070
:100bc000819120001000200098030700381c0700c6
:100bd000400798004e009000e10f500003003a00db
:100be00040202b001007980002003700b0202b0097
:100bf000100798004e0090000000e0000300320053
:100c000020212b00000f78000200370050212b001c
:100c1000000f78001e007800801f78009e00900072
:100c2000811f780030232b00801f780080912000e6
:100c30008d070700e68757008191200010002000f3
:100c40007a030700421b070020079800310798002d
:100c50002e019000be019000807020000100200055
:100c6000800f5100818f590003003a0040202b0073
:100c70001007980002003700b0202b0010079800e2
:100c80002e009000be009000809fbe009e0090004d
:100c9000811f7800d0242b00801f780080912000d5
:100ca00071070700e887570081912000100020009d
:100cb0005e0307004e1b07002007980031079800cd
:100cc0002e019000be019000002f2d000100200099
:100cd000800f5100818f590003003a0040202b0003
:100ce0001007980002003700b0202b001007980072
:100cf0002e009000be009000809fbe009e009000dd
:100d0000811f7800c0262b00801f78008091200072
:100d100055070700e8875700819120001000200048
:100d2000420307003d220700200798003107980082
:100d30002e019000be019000e00120000100200083
:100d4000800f5100818f590003003a0040202b0092
:100d50001007980002003700b0202b001007980001
:100d60002e009000be009000809fbe009e0090006c
:100d7000811f7800b0282b00801f78008091200010
:100d800039070700e88757008191200010002000f4
:100d90002603070015220700200798003107980056
:100da0002e019000be0190002000200001002000d4
:100db000800f5100818f590003003a0040202b0022
:100dc0001007980002003700b0202b001007980091
:100dd0002e009000be009000809fbe009e009000fc
:100de000811f7800902a2b00801f780080912000be
:100df0001d070700e88757008191200010002000a0
:100e00000a030700d71b0700200798003107980046
:100e10002e019000be019000c012200001002000b1
:100e2000800f5100818f590003003a0040202b00b1
:100e30001007980002003700b0202b001007980020
:100e40002e009000be009000809fbe009e0090008b
:100e5000811f7800802c2b00801f7800809120005b
:100e600001070700e887570081912000100020004b
:100e7000ee0207000f1b07002007980031079800bb
:100e80002e019000be01900080072000010020008c
:100e9000800f5100818f590003003a0040202b0041
:100ea0001007980002003700b0202b0010079800b0
:100eb0002e009000be009000809fbe009e0090001b
:100ec000811f7800702e2b00801f780080912000f9
:100ed000e5060700e88757008191200010002000f8
:100ee000d2020700241b0700200798003107980052
:100ef0002e019000be019000001e20000100200085
:100f0000800f5100818f590003003a0040202b00d0
:100f10001007980002003700b0202b00100798003f
:100f20002e009000be009000809fbe009e009000aa
:100f3000811f780060302b00801f78008091200096
:100f4000c9060700e88757008191200010002000a3
:100f5000b60207000000eb000080fa000000060067
:100f60000200fa00000f7800100020000a1b0700a2
:100f700010002000321b070020002000010020008c
:100f800045210700e001200001002000702107003a
:100f9000002f2d0001002000751a0700807020002e
:100fa000010020004a1a0700c012200001002000a2
:100fb000431b07008007200001002000941a07004f
:100fc000001e200001002000c21a07000000eb00f4
:100fd0000080fa00000006000200fa00000f78000e
:100fe00051322b0010002000900207001100200059
:100ff00010002000e41c07000000eb000080fa0055
:10100000000006000200fa00000f780071332b0088
:1010100010002000850207008000eb001000200077
:10102000d91c07000000eb000080fa000000060059
:101030000200fa00000f7800a1342b0010002000fd
:101040007a0207001100200020002000ce1c0700bb
:101050000000eb000080fa00000006000200fa0029
:10106000000f780051352b00100020006f020700a0
:101070008000eb0020002000c31c07000000eb00f4
:101080000080fa00000006000200fa00000f78005d
:1010900011362b0010002000640207001100200010
:1010a00030002000b81c07000000eb000080fa00b0
:1010b000000006000200fa00000f780001372b0044
:1010c00010002000590207008000eb0030002000d3
:1010d000ad1c07000000eb000080fa0000000600d5
:1010e0000200fa00000f780001382b0010002000e9
:1010f0004e020700110020000000eb00a21c0700b8
:101100000000eb000080fa00000006000200fa0078
:10111000000f7800c1382b001000200043020700a8
:101120008000eb000000eb00971c07000000eb00c4
:101130000080fa00000006000400fa00000f7800aa
:1011400010002000941a07000000e00006003200a2
:1011500091392b0010002000340207000000eb0042
:101160001007980005003700813a2b00100020007e
:101170002e0207000000eb00100798001e009000f0
:101180000080fa00000006000400fa00000f78005a
:101190000000eb00801a07000000e00006003200ab
:1011a000b13c2b0010002000200207000000eb00e3
:1011b0001007980005003700813a2b00100020002e
:1011c0001a0207000000eb00100798001e009000b4
:1011d0000080fa00000006000400fa00000f78000a
:1011e00010002000961a07000000e0000600320000
:1011f000b13d2b00100020000c0207000000eb00a6
:101200001007980005003700813e2b0010002000d9
:10121000060207000000eb00100798001e00900077
:101220000080fa00000006000400fa00000f7800b9
:101230000000eb00821a07000000e0000600320008
:1012400061402b0010002000f80107000000eb00b7
:10125000100798000500370041412b0010002000c6
:10126000f20107000000eb00100798001e0090003c
:101270000080fa00000006000200fa00000f78006b
:1012800031432b0010002000e8010700d4180700ac
:101290000000eb000080fa00000006000200fa00e7
:1012a000000f7800b1432b0010002000df01070081
:1012b0000000eb000080fa00000006000200fa00c7
:1012c000000f780031442b0010002000d7010700e8
:1012d0000000eb000080fa00000006000200fa00a7
:1012e000000f7800b1442b0010002000cf01070050
:1012f0000000eb000080fa00000006000200fa0087
:10130000000f780031452b0010002000c7010700b6
:101310000000eb000080fa00000006000600fa0062
:1013200020079800a20020008000eb002e00900013
:10133000de050700008fbe001e00be006419070016
:101340000000eb000080fa00000006000600fa0032
:1013500020079800a20020008000eb002e009000e3
:10136000d2050700008fbe001e00be0080190700d6
:101370000000eb000080fa00000006000600fa0002
:1013800020079800a20020008000eb002e009000b3
:10139000c6050700008fbe001e00be006c200700bf
:1013a0000000eb000080fa00000006000600fa00d2
:1013b00020079800a20020008000eb002e00900083
:1013c000ba050700008fbe001e00be0032200700d5
:1013d0000000eb000080fa00000006000600fa00a2
:1013e00020079800a20020008000eb002e00900053
:1013f000ae050700008fbe001e00be00301a0700b9
:101400000000eb000080fa00000006000600fa0071
:1014100020079800a20020008000eb002e00900022
:10142000a2050700008fbe001e00be00781907004d
:101430000000eb000080fa00000006000600fa0041
:1014400020079800a20020008000eb002e009000f2
:1014500096050700008fbe001e00be009d19070004
:101460000000eb000080fa00000006001400fa0003
:10147000000f98008e80e8000000eb0080087800e4
:101480008e80e8000000eb00900098008e80e8005d
:101490000000eb00a00098008e80e8000000eb0048
:1014a000b00098008e80e8000000eb00c0009800bb
:1014b0008e80e8000000eb00d00098008e80e800ed
:1014c0000000eb00e00098000e80e800660040009d
:1014d000801f78000e80e800801f78000e80e800f2
:1014e0000080e800801f78000e80e8006400400063
:1014f000801f78000e80e8006c004000801f78009c
:101500000e80e80068004000801f78000e80e80030
:101510006a004000801f7800a0452b00801f7800e3
:101520000e08900001060700f0875700000f7800b2
:10153000600020009e0f10000c003c00f1462b00c4
:10154000100020003901070011482b001000200076
:1015500036010700014a2b0010002000330107006c
:101560000000eb00100f9800740037000e80e800b8
:10157000500090000000e000040034000e80e800fd
:1015800050009000ec0f500006003400614c2b001e
:1015900010002000250107000000eb00100f98004c
:1015a000660037000e80e800400090000000e00078
:1015b000040034000e80e80040009000ff0f50004f
:1015c00006003400914e2b00100020001701070088
:1015d0000000eb00100f9800580037000e80e80064
:1015e00060009000ea0f5000050034000e80e80013
:1015f000e000900030062000808f5000060034008c
:10160000a1502b0010002000080107000000eb0093
:10161000100f9800490037000e80e800200090006d
:101620000000e000040035000e80e800200090007b
:10163000f70f500006003400e1522b00100020008c
:10164000fa0007000000eb00100f98003b00370085
:101650000e80e800100090000000e000050035005a
:101660000e80e80090009000b0032000808f5000b2
:101670000600340021552b0010002000eb0007006d
:101680000000eb00100f98002c0037000e80e800df
:10169000100078000000e000050035000e80e80032
:1016a00090007800b0032000808f500006003400c6
:1016b00081572b0010002000dc0007000000eb0029
:1016c000100f98001d0037000e80e80030009000d9
:1016d0000000e000040034000e80e80030009000bc
:1016e000e70f500006003400e1592b0010002000e5
:1016f000ce0007000000eb00100f98000f0037002d
:101700000e80e800371d070080912000a71d07000c
:10171000f15b2b0010002000c40007008191200025
:1017200010002000c100070041132b001000200012
:10173000be0007000000eb00100f98001e0890008c
:081740000080fa000000060021
:020000040000fa
:1075a4000000fa00809e20000b070700809e200048
:1075b4005b070700e09d200007070700e09d20000f
:1075c40057070700209f200003070700209f200083
:1075d400530707000080fa00000006004600fa0086
:1075e400c17a2b00100020000fe90700504e8000e4
:1075f400202798002e219000e30f5100260032002e
:10760400ae219000e38f51000a003c002e20900030
:10761400e10f5000180032002e219000e10f5100bc
:1076240019003c00ae2190000300e0000e0032007f
:107634002d0037002e209000e50f50001e00320070
:107644002e219000e50f510017003500ae21900067
:10765400e68f51001c0032002e209000e70f5000ee
:107664001d00320020003700e17b2b0010002000b9
:10767400ede807001f003700817c2b00100020007c
:10768400e9e807001b003700517d2b0010002000a3
:10769400e5e8070017003700f17d2b0010002000fb
:1076a400e1e8070013003700917e2b001000200052
:1076b400dde807000f003700217f2b0010002000b9
:1076c400d9e807000b003700c17f2b001000200011
:1076d400d5e807000700370091802b001000200038
:1076e400d1e807000300370081812b00100020003f
:1076f400cde8070001822b0010002000cae8070033
:10770400809e2000c8060700823e2000030020005f
:1077140023f70700008fbe00e40047001e01be00ef
:10772400829fbe0050822b00801f780001007800e9
:10773400ccec0700e6875700e40047001000200067
:10774400b9e80700405180000000e0000400320066
:1077540021842b0010002000b3e807000300370049
:10776400a1852b0010002000afe80700604e8000c8
:107774000000e0000400320031872b0010002000dc
:10778400a9e8070003003700d1882b00100020006f
:10779400a5e80700818a2b0010002000a2e807005a
:1077a400209f2000a0060700823e20000300200046
:1077b400fbf60700008fbe00e40047001e01be0078
:1077c400829fbe00b08a2b00801f780001007800e1
:1077d400a4ec0700e6875700e400470010002000ef
:1077e40091e80700705180000000e00004003200be
:1077f400718c2b00100020008be807000300370079
:10780400e18d2b001000200087e80700704e8000f7
:107814000000e00004003200618f2b001000200003
:1078240081e8070003003700e1902b0010002000de
:107834007de80700818a2b00100020007ae8070009
:107844000080fa00000006000200fa00000f780031
:107854009e007800618060000004e00001003200b6
:10786400530607001e0078000000d100610060008c
:107874000004e00001003200b50107001e0078009a
:107884004200de00610060000004e00001003200fc
:107894003b0107001e0078004300de006100600029
:1078a4000004e00001003200db0107001e00780044
:1078b4004400de00610060000004e00001003200ca
:1078c400200207000080fa00000006000400fa000d
:1078d400008fbe001e00be00205188003151880078
:1078e400225180003351800000902000d1032000f9
:1078f400800f5100818f5900040036000090200051
:10790400d103200020518800315188002651800085
:107914003751800086007800803e20000009b800be
:107924006030b9000302780000024200803e20006b
:1079340000b8b90000024200840178002251880096
:10794400335188000080fa00000006000000fa00ad
:107954002051800031518000823e2000030020002d
:107964008ff607000080fa00000006000400fa0009
:10797400008fbe001e00be00005188001151880017
:10798400025180001351800000902000d103200098
:10799400800f5100818f59000400360000902000b0
:1079a400d103200000518800115188000651800045
:1079b4001751800086007800803e20000009b8003e
:1079c4006030b9000302780000024200803e2000cb
:1079d40000b8b90000024200840178000251880016
:1079e400135188000080fa00000006000000fa002d
:1079f4000051800011518000823e200003002000cd
:107a040067f607000080fa00000006000400fa0090
:107a1400008fbe001e00be00805188009151880076
:107a24008051800091518000e00f5000e08f580099
:107a340004003a001000200001002000805188005a
:107a4400915188008251800093518000800c200065
:107a540001002000800f5100818f5900040036007e
:107a6400800c200001002000805188009151880082
:107a7400865180009751800086007800803e200067
:107a84000009b8006030b900030278000002420027
:107a9400803e200000b8b900000242008401780052
:107aa40082518800935188000080fa00000006008b
:107ab4000000fa008051800091518000823e200035
:107ac4000300200036f607000080fa0000000600dc
:107ad4000400fa00008fbe001e00be00a051880002
:107ae400b1518800a0518000b1518000e00f5000d6
:107af400e08f580004003a0010002000010020002c
:107b0400a0518800b1518800a2518000b351800077
:107b140000902000d1032000800f5100818f590074
:107b24000400360000902000d1032000a0518800fa
:107b3400b1518800a6518000b751800086007800ba
:107b4400803e20000009b8006030b90003027800cc
:107b540000024200803e200000b8b900000242004a
:107b640084017800a2518800b35188000080fa0093
:107b7400000006000000fa00a0518000b15180000e
:107b8400823e20000300200005f607000080fa0072
:107b9400000006000200fa00000f78001e00e0005a
:107ba400100032001000200040518800809e200008
:107bb400910507000000eb00604e8800504e8000e5
:107bc400e70f500016003a008000eb000000eb00c5
:107bd400ec0107008000eb0020002000e901070011
:107be4000f0037000000eb0040518800809e200009
:107bf400810507000000eb00604e8800504e8000b5
:107c0400e70f500006003a008000eb000000eb0094
:107c1400dc0107008000eb0020002000d9010700f0
:107c2400100020000080fa00000006000000fa00a6
:107c3400405180000080fa00000006000200fa00b3
:107c4400000f78001e00e000110032001000200038
:107c540070518800209f2000670507001000200055
:107c6400704e8800504e8000e70f50000c003a0020
:107c7400110020000000eb00c201070011002000e9
:107c840020002000bf010700640107000400370042
:107c94000000eb00705188000000eb00704e88007b
:107ca400100020000080fa00000006000000fa0026
:107cb400705180000080fa00000006000400fa0001
:107cc400008fbe001e00be00505188006151880024
:107cd4005051800061518000e00f5000e08f580047
:107ce40004003a00100020000100200050518800d8
:107cf400615188005251800063518000009020003f
:107d0400d1032000800f5100818f590004003600f8
:107d140000902000d1032000505188006151880058
:107d2400565180006751800086007800803e200014
:107d34000009b8006030b900030278000002420074
:107d4400803e200000b8b90000024200840178009f
:107d540052518800635188000080fa000000060038
:107d64000000fa005051800061518000823e2000e2
:107d7400030020008af507000080fa0000000600d6
:107d84000000fa00504e8000e70f50006e003200f1
:107d9400504e80000000e00006003a00209d2000c4
:107da4000d050700209d20005d0507001000200040
:107db400504e8800504e8000e10f50000c003a00f5
:107dc400209d2000180507000001be0020518000fe
:107dd40031518000800f5100818f59005a003900c1
:107de400209d20000405070020002000504e88003c
:107df400504e8000e20f500005003a0011002000b0
:107e0400300020005f01070030002000504e880041
:107e1400504e8000e30f50000f003a00209d2000d8
:107e2400010507000001be00703e20000100200093
:107e3400800f5100818f590043003600110020004b
:107e4400100020004f010700209d2000ea040700d5
:107e540040002000504e8800504e8000e40f500037
:107e64000c003a00209d2000ef0407000001be0032
:107e7400f0a52e0001002000800f5100818f5900d1
:107e840031003600209d2000db0407005000200054
:107e9400504e8800405180000000e0000500320090
:107ea400209d2000d404070070002000504e88005c
:107eb40025003700504e8000e50f500010003a00b6
:107ec400209d2000d80407000001be00703e200061
:107ed40001002000800f5100818f59001a003600e4
:107ee400110020000000eb0026010700cb00070072
:107ef400209d2000c004070060002000504e880030
:107f0400504e8000e60f50000f003a00209d2000e4
:107f1400c50407000001be00703e200001002000df
:107f2400800f5100818f5900070036001100200096
:107f34002000200013010700209d2000ae0407004c
:107f440070002000504e88000080fa0000000600f7
:107f54000000fa00e09d2000b30407000001be0009
:107f64000051800011518000800f5100818f590011
:107f7400270039000051800011518000e00f5000ab
:107f8400e08f580001003a00210037000000eb00a8
:107f9400405188000000eb00604e8800809e200065
:107fa400950407000000eb00705188008000eb008e
:107fb4000000eb00f3000700ad000700401f2000a5
:107fc400110507008000eb0030002000ed000700e1
:107fd400400620000c0507008000eb001000200084
:107fe400e800070040062000070507008000eb00ba
:107ff40020002000e30007004006200002050700df
:10800400e09d2000dc040700e09d20007a040700c6
:108014000080fa00000006006200fa00190507005b
:10802400000f7800e04e80009e0f100026003600fe
:108034001e007800e04e8800405180000000e000ff
:108044000e003200504e8000e70f50000b003a0043
:1080540010002000604e8800809e20006604070007
:10806400110020000000eb00c600070011002000f2
:1080740020002000c300070068000700200420003f
:108084000e004000000407008e80e8002004200059
:108094000e004000801f78001e007800801f7800ca
:1080a40070922b00801f7800010078006dea0700b1
:1080b400e68757008e80e800100020005ae607008b
:1080c4000e80e800de090700405180000000e00057
:1080d4001a003200504e8000e70f500017003a009b
:1080e400604e80000000e00014003200809e2000fa
:1080f4004d0407000001be00505180006151800012
:10810400800f5100818f59000c0036000000eb00f5
:10811400604e8800704e80000000e00007003a00c6
:108124008000eb000000eb00960007008000eb00ed
:1081340020002000930007004d0007000080fa0093
:10814400000006000000fa00705180000000e0000a
:1081540030003200504e8000e70f50002d003a00ee
:10816400704e80000000e00017003200209f2000c5
:108174002d0407000001be00805180009151800051
:10818400800f5100818f5900220036000000eb005f
:10819400704e8800209f200017040700604e800066
:1081a4000000e0001b003a008000eb000000eb0040
:1081b400740007008000eb0020002000710007001d
:1081c4002b00070013003700209f2000160407002f
:1081d4000001be00a0518000b1518000800f510009
:1081e400818f59000b00360010002000704e88006b
:1081f400209f200000040700110020000000eb0075
:108204006000070011002000200020005d0007002e
:10821400020007000080fa00000006006000fa0077
:10822400804e80000000e800804e8800000420009a
:108234000e00400094030700814e800000042000db
:108244000e004000801f7800811f7800e0932b000f
:10825400801f78000e00780002ea0700e6875700c6
:108264000e007800760907000080fa00000006007e
:108274006000fa00000420000e00400082030700a2
:10828400814e8000000420000e004000801f780012
:10829400811f780040952b00801f78000e00780025
:1082a400f0e90700e68757000e007800640907002c
:1082b4000080fa00000006000000fa00c922a900ac
:1082c400d0c2a900d0e2a900d102a900d122a900fc
:1082d400c942a900c962a900c982a900d042a90063
:1082e400d022a900d002a900c862a900c842a900ee
:1082f400c9e2a900c9c2a900c9a2a90000000000de
:10830400cd22a90000000000d4c2a9000000000092
:10831400d4e2a90000000000d502a900000000007a
:10832400d522a90000000000cd42a90000000000f1
:10833400cd62a90000000000cd82a9000000000069
:10834400d442a90000000000d422a90000000000cb
:10835400d402a90000000000cc62a90000000000c3
:10836400cc42a90000000000cde2a90000000000fa
:10837400cdc2a90000000000cda2a9000080fa002f
:10838400000006000800fa00000f780011079800aa
:108394001e0090000000e0000200320010002000e7
:1083a40010079800000000001e0078006101b90069
:1083b4002207980033079800f000200001002000f5
:1083c4002e019000be019000800f5100818f590052
:1083d400ba003e002e009000be0090000060010034
:1083e4000f00370019003700230037002a00370038
:1083f400330037003d003700470037005100370095
:108404005b003700650037006f00370078003700e5
:10841400820037008c003700930037009d0037003e
:108424001e00900061406000614060000041400017
:10843400d12c200091407800d0cfb30000c0600060
:1084440002407000cde2b7009c0037001e0090008f
:1084540061406000614060004601dd00412d200064
:1084640091407800f0cbb30000c06000024070007f
:10847400d4e2b700910037001e0090006140600014
:10848400c700dd00d4c2bf000074a1000140700029
:10849400d4e2b700890037001e00900061406000fc
:1084a40061416000512d200091407800e0cfb3007d
:1084b40000c0600002407000d5e2b7007f003700c2
:1084c4001e00900061406000614060000041400077
:1084d400512d200091407800d0cfb30000c060003f
:1084e40002407000d5e2b700740037001e0090000f
:1084f40061406000614060004201dd00d12c200039
:1085040091407800b0cfb30000c06000024070001a
:10851400cde2b700690037001e00900061406000a2
:10852400614060004301dd00d12c200091407800bf
:1085340070cfb30000c0600002407000cde2b7000d
:108544005e0037001e0090006140600061406000e2
:108554004401dd00d12c200091407800f0ceb3001e
:1085640000c0600002407000cde2b7005300370045
:108574001e00900061406000614060004201dd0027
:10858400412d200091407800b0cfb30000c06000be
:1085940002407000d4e2b700480037001e0090008b
:1085a400614060006140600000414000412d2000b6
:1085b40091407800d0cfb30000c06000024070004a
:1085c400d4e2b7003d0037001e0090006140600017
:1085d40061416000412d200091407800e0cfb3005c
:1085e40000c0600002407000d4e2b70033003700de
:1085f4001e00900061406000614060004301dd00a6
:10860400c12c20009140780070cfb30000c06000fe
:1086140002407000cce2b700280037001e00900032
:1086240061406000614060004201dd00c12c200017
:1086340091407800b0cfb30000c0600002407000e9
:10864400cce2b7001d0037001e00900061406000be
:10865400c700dd00cdc2bf000074a100014070005e
:10866400cde2b700150037001e00900061406000a5
:10867400614060004601dd00d12c2000914078006b
:10868400f0cbb30000c0600002407000cde2b70040
:108694000a0037001e0090006140600061406000e5
:1086a4004501dd00d12c200091407800f0cdb300cd
:1086b40000c0600002407000cde2b7000080fa0004
:1086c400000006000800fa00000f78000000000017
:1086d4000000eb00605288001e0078006101b900c0
:1086e4002207980033079800f000200001002000c2
:1086f4002e019000be019000800f5100818f59001f
:108704007d003e002e009000be009000006001003d
:108714000f003700150037001b003700200037001a
:10872400240037002a0037003000370036003700b5
:108734003c00370042003700480037004c00370047
:1087440052003700580037005d00370063003700df
:10875400cdc2bf000080fb000000d100614060007a
:108764000080fb001007980065003700d4c2bf00ea
:108774000080fb004600de00614060000080fb00da
:10878400100798005e003700d4c2bf000080fb00d1
:108794004700de000080fb001007980058003700f7
:1087a400d5c2bf00614060000080fb001007980044
:1087b40053003700d5c2bf000080fb000000d10089
:1087c400614060000080fb00100798004c003700f7
:1087d400cdc2bf000080fb004200de0061406000ab
:1087e4000080fb001007980045003700cdc2bf0091
:1087f4000080fb004300de00614060000080fb005d
:10880400100798003e003700cdc2bf000080fb0077
:108814004400de00614060000080fb001007980007
:1088240037003700d4c2bf000080fb004200de00e6
:10883400614060000080fb001007980030003700a2
:10884400d4c2bf000080fb000000d1006140600082
:108854000080fb001007980029003700d4c2bf0035
:10886400614060000080fb0010079800240037007e
:10887400ccc2bf000080fb004300de00614060000a
:108884000080fb00100798001d003700ccc2bf0019
:108894000080fb004200de00614060000080fb00bd
:1088a4001007980016003700cdc2bf000080fb00ff
:1088b4004700de000080fb0010079800100037001e
:1088c400cdc2bf000080fb004600de0061406000b6
:1088d4000080fb001007980009003700cdc2bf00dc
:1088e4000080fb004500de00614060000080fb006a
:1088f40010079800020037008000eb001107980071
:108904001e0090000080fa00000006000600fa0035
:108914002007980010002000000f78000000eb00f2
:10892400100798000b0037002e0090001e00600016
:10893400800078001e00900092fe07001e00780060
:1089440000004000000f78001e0090000000e800c6
:10895400100798001e009000ef0f5000f2ff340043
:108964000080fa00000006000600fa001000200053
:10897400100798000000eb00000f78000000eb00e7
:10898400200798000c0037002e0090004dff0700d0
:108994000000e000020032001e0090001e0f4000a4
:1089a4001e00900000004000100798002e00900068
:1089b4000000e800200798002e009000ef0f500000
:1089c400f1ff34001e0078000080fa000000060069
:1089d4000800fa00000f7800000000000000eb001f
:1089e400605288001e0078006101b90022079800d7
:1089f40033079800f0002000010020002e019000b1
:108a0400be019000800f5100818f59004a003e0042
:108a14002e009000be009000006001000f0037009f
:108a2400140037001a0037001c0037001e003700fe
:108a340020003700220037002400370026003700ca
:108a4400280037002a0037002c0037002e0037009a
:108a5400300037003200370034003700c2c2bf0094
:108a64000080fb004700de000080fb001007980038
:108a740033003700c3c2bf000080fb004200de00a9
:108a8400614060000080fb00100798002c00370054
:108a9400615280001107980029003700625280005b
:108aa40012079800260037006352800013079800cd
:108ab4002300370060528000100798002000370020
:108ac40061528000110798001d0037006252800037
:108ad400120798001a0037006352800013079800a9
:108ae4001700370060528000100798001400370008
:108af4006152800011079800110037006252800013
:108b0400120798000e003700635280001307980084
:108b14000b003700605280001007980008003700ef
:108b240061528000110798000500370062528000ee
:108b340012079800020037008001eb001307980029
:108b44001e0090000080fa00000006000600fa00f3
:108b540010002000100798000000eb00000f7800c0
:108b64000000eb00200798000c0037002e00900056
:108b740097ff07000000e000020032001e00900092
:108b84001e0f40001e0090000000400010079800d7
:108b94002e0090000000e800200798002e009000ae
:108ba400ef0f5000f1ff34001e0078000080fa003f
:048bb40000000600b7
:020000040000fa
:101748000200fa000000eb00000f780027003700c5
:101758009e0178001e0078004700dd0080007800b8
:10176800408120000080400000017800c318dd009f
:101778004080200000804000020878001e007800a9
:101788004300dd008080e800408020008080400029
:101798000000eb00800878001e0078004300dd00a0
:1017a800e400400040802000808040000000eb0002
:1017b800800878001e0078004300dd00e600400045
:1017c8004080200080804000f007200080087800da
:1017d8001e0078008000400040912000808040007a
:1017e8000000eb00800878001e0fe80010002000c1
:1017f8009e0f1000d6ff34007001200040118800b1
:1018080021e2a80020a2a9002062a900004020002f
:10181800101188008560a9008580a900910a200020
:1018280091407800f0c8b30000c0600001c6b30062
:1018380001407000a9e0b700a10a2000914078009b
:1018480080cfb30000c060000014a000aae0b70079
:101858009560a8009580a90070012000c01188003b
:1018680031e2a80030a2a9003062a900004020009f
:101878009011880087c0a90087e0a900310b2000db
:101888009140780080cfb30000c060006040b30092
:10189800b3e0b700310b200091407800f0c8b300e6
:1018a80000c0600001c2b30001407000b3e0b7009f
:1018b80097c0a80097e0a9000080fa000000060081
:1018c8000a00fa0010079800210798001e009000ef
:1018d800400798004e009000e10f500009003200c8
:1018e8004e009000e20f500006003200ae0090005b
:1018f8000040eb00804878000000eb0030079800bb
:101908000d0037009c0107001e0090004300dd0019
:1019180080007800408020006800500080804000ef
:101928002e009000d1250700000f78009c010700c9
:101938001e007800300798003e0090000080fa00f2
:10194800000006000c00fa001007980041479800b4
:101958001e009000400798004e009000e10f5000d4
:10196800040032004e009000e20f500008003200e0
:101978000e00370023c2bf000080fb000000d1002a
:10198800614060000080fb00000f7800090037000c
:1019980033c2bf000080fb000000d100614060003e
:1019a8000080fb00000f78000200370010002000c4
:1019b800000f78001e00e00015003a001e0090009d
:1019c800500798005e009000e10f500004003200bc
:1019d8005e009000e20f5000070032000c00370054
:1019e8004e4090000080fb0020118800100020006d
:1019f80030079800080037004e4090000080fb0038
:101a0800a01188001000200030079800020037005d
:101a18000000eb00300798003e0090000080fa00bc
:101a2800000006000600fa00100798002107980039
:101a38000000eb00000f78000b0037001e00780054
:101a4800800078002e009000008040001040780050
:101a5800804078001e009000baff07000000e000f8
:101a6800010032001e0fe8001e0078008000780098
:101a78002e00900000804000104078000004e00034
:101a8800eeff3a000000eb000080fa0000000600bc
:101a98000800fa00100798001e0090003007980010
:101aa8003e009000e10f5000060032003e0090001a
:101ab800e20f5000030032000000eb0020079800fe
:101ac8000c0037002c0107001e0090004300dd00c9
:101ad80080007800408020006800500000804000ae
:101ae8008e250700000f78002d0107001e007800e2
:101af800200798002e0090000080fa0000000600e1
:101b08000600fa00100798001e00900020079800b1
:101b18002e009000e10f5000040032002e009000cb
:101b2800e20f5000080032000e00370023c2bf0049
:101b38000080fb000000d100614060000080fb00d5
:101b4800000f78000900370033c2bf000080fb0097
:101b58000000d100614060000080fb00000f7800a9
:101b68000200370010002000000f78001e007800e7
:101b78000080fa00000006000600fa00000f780056
:101b88001e007800200798002e009000e10f5000fa
:101b9800060032002e009000e20f500003003200d1
:101ba8000000eb0010079800060037001e00e9004f
:101bb8008000400040912000008040001000780024
:101bc800100798001e0090000080fa000000060030
:101bd8000400fa00000f78001e0078001007980033
:101be8001e009000e10f5000040032001e0090001b
:101bf800e20f500001003200060037001e00e90025
:101c08008000400040912000808040000000eb00f0
:101c1800800878000080fa00000006000800fa003a
:101c2800100798001e009000200798002e009000d2
:101c3800e10f5000040032002e009000e20f500027
:101c4800010032001f003700cb0007001e00900083
:101c58004300dd00800078004080200068005000cc
:101c680000804000232507001e00900030079800e0
:101c78003e009000e10f5000060032003e00900048
:101c8800e20f50000a0032000d00370030118000ca
:101c9800000f780022c2bf00614060000004e0002d
:101ca800faff3a0006003700b0118000000f7800f4
:101cb80032c2bf00614060000004e000faff3a0051
:101cc800b70007000080fa00000006000400fa00d0
:101cd800000f78001e007800100798001e00900082
:101ce800e10f5000040032001e009000e20f500087
:101cf80006003200090037002342a9000000000056
:101d08002342a80000000000040037003342a90065
:101d1800000000003342a800000000000080fa0024
:101d280000000600809fbe000000fa00004080000e
:101d38001140800061004000e080480000408800b9
:101d4800114088008580a9000080fa004f00be007d
:101d580000400600809fbe000000fa001600370011
:101d6800304080008000e8005040800080806000a3
:101d780040408000808f500005003a0030118000fc
:101d8800a048880010002000a04888000a003700fa
:101d98002140800030408000808040003011800069
:101da80080487800304080008000e8005040800083
:101db800008060003040880022c2bf00614060009f
:101dc8000004e000e6ff3a008560a9000080fa0000
:101dd8004f00be0000400600809fbe000000fa00d1
:101de800004080001140800061004000e080480011
:101df800004088001140880087e0a9000080fa00b0
:101e08004f00be0000400600809fbe000000fa00a0
:101e180016003700704080008000e8009040800085
:101e28008080600080408000808f500005003a006c
:101e3800b0118000b048880010002000b048880029
:101e48000a003700614080007040800080804000b8
:101e5800b011800080487800704080008000e80061
:101e680090408000008060007040880032c2bf004f
:101e7800614060000004e000e6ff3a0087c0a90066
:0c1e88000080fa004f00be000040060081
:020000040000fa
:108bb8000000fa0010002000e5e40700e0082000ab
:108bc800cee407000000eb00cce407000000eb0057
:108bd800dfe407000080fa00000006000400fa0045
:108be8001007980010002000d9e4070000082000b2
:108bf800c2e407001e009000100078003b01070047
:108c0800004f78001e80fb00bce407001e009000a7
:108c18001000900035010700004f78001e80fb000f
:108c2800b6e407001e009000200090002f01070006
:108c3800004f78001e80fb00b0e407001e00900083
:108c480030009000ade407001e0090004000900046
:108c580026010700004f78001e80fb00a7e40700ec
:108c68001e0090005000900020010700004f78007f
:108c78001e80fb00a1e407001e0090006000900029
:108c88001a010700004f78001e80fb009be40700d4
:108c98000000eb00aee407000000eb000080fa00e3
:108ca800000006000400fa001007980010002000d9
:108cb800a7e407000000eb0090e40700500520003f
:108cc8008ee40700004f78001e4078001a01070064
:108cd8008080fb001e0090000108780050052000ed
:108ce80086e40700004f78001e4078001201070054
:108cf8008080fb001e0090001100980050052000a5
:108d08007ee40700004f78001e4078000a01070043
:108d18008080fb001e009000210098005005200074
:108d280076e40700800078001e009000310098006b
:108d38005005200071e40700004f78001e407800bd
:108d4800fd0007008080fb001e0090004100980095
:108d58005005200069e40700004f78001e407800a5
:108d6800f50007008080fb001e009000510098006d
:108d78005005200061e40700004f78001e4078008d
:108d8800ed0007008080fb001e0090006100980045
:108d98000000eb006ee407000000eb000080fa0022
:108da800000006005600fa00702798000e007800b0
:108db800bcff07003e009000002f98008e2890000e
:108dc800e48f5000290032000e299000e40f510072
:108dd8000a003c008e299000e28f510017003200f3
:108de8000e289000e20f50001a003c008e289000d8
:108df800e18f50000b003200340037000e2990003c
:108e0800e60f5100250032008e299000e68f5100b0
:108e18001c0035000e289000e70f50002500320096
:108e28002a0037007e209000e1a02b0004000900f2
:108e3800315878005000b100290037007e2090009a
:108e480032a12b0004000900325878005000b1000c
:108e5800230037007e20900083a12b000400090026
:108e6800335878005000b1001d0037007e20900074
:108e7800d1a12b0004000900315878005000b1003e
:108e8800170037007e20900022a22b000400090062
:108e9800325878005000b100110037007e20900051
:108ea80073a22b0004000900335878005000b10069
:108eb8000b0037007e209000c1a22b00040009009f
:108ec800315878005000b100050037007e2090002e
:108ed80012a32b0004000900325878005000b1009a
:108ee8005e0090006101b9000080eb008080eb001b
:108ef8000201400083814800122f9800232f980018
:108f0800b0002000010020001e299000ae2990002a
:108f1800800f5100818f59003f003e001e289000ad
:108f2800ae289000006001000b0037000e003700eb
:108f38001100370014003700170037001a003700f7
:108f48001d003700200037002300370026003700b7
:108f5800290037002c00370061a32b007e209000e9
:108f68008ee707002f003700b1a32b007e2090006a
:108f78008ae707002b00370001a42b007e20900011
:108f880086e707002700370051a42b007e209000b9
:108f980082e7070023003700a1a42b007e20900061
:108fa8007ee707001f003700f1a42b007e20900009
:108fb8007ae707001b00370041a52b007e209000b0
:108fc80076e707001700370091a52b007e20900058
:108fd80072e7070013003700e1a52b007e20900000
:108fe8006ee707000f00370031a62b007e209000a7
:108ff8006ae707000b00370081a62b007e2090004f
:1090080066e7070007003700d1a62b007e209000f6
:1090180062e707000300370011a32b007e209000b1
:109028005ee70700ee009000007d20000080400011
:109038009e0078001e019000ae0190004e02900044
:10904800ee024700801f7800811f7800821f780099
:10905800831f7800841f780020a72b00801f7800ca
:10906800050078007ee60700ec875700ee00470011
:109078007e20900049e707000000eb000080fa001e
:10908800000006001000fa00700798000e00780033
:1090980004ff07001e0178009e0190002e02900038
:1090a800ee009000007d200000804000ce0090007f
:1090b800de029000821f7800831f7800841f7800ea
:1090c800801f7800811f7800851f780070a82b000a
:1090d800801f78007e00900061e60700ee87570049
:1090e8000000eb000080fa00000006000400fa000f
:1090f800204798002e4090000080fb00a20020002e
:10910800110009000280d8004400dd00004f7800fb
:109118002e4090000080fb00a200200011000900f2
:109128000280d8008000fd001e4f40001e80fb001a
:109138000080fa00000006000400fa0020479800aa
:109148002e4090006f4f60002e4090008080fb0002
:10915800000f2000008060004480de006a00b90033
:10916800804078001e40780000c04000004f780022
:109178001e80fb000080fa00000006000000fa00d4
:109188000000eb00800888000000eb003008880031
:10919800f0ff28006008880084e0a90094e0a80097
:1091a80011e1a8000080fa00000006000000fa00a3
:1091b8002b0107000080fa00000006000200fa00f8
:1091c800000f78001e007800100078000080fa0078
:1091d800000006000200fa00000f78001e00780068
:1091e800640007001e007800020007000080fa00f3
:1091f800000006000200fa00000f78001e01780047
:109208006000b800300198004101980096000700fe
:109218001e01780010019800210198000080fa00d2
:10922800000006000600fa00200798008e000700dc
:10923800008fbe002e009000100078000000e000b3
:10924800230032002e009000a00090001000900033
:10925800be0f5000ae8f58000f0036002e00900051
:1092680030019000c00190002e009000a0009000f6
:10927800100090003e024000ae8248000400be008c
:1092880002004000838048002e01900030019800c1
:10929800410198000e0037002e0090003001900028
:1092a800c00190002e009000a000900010009000d7
:1092b8003e021000ae8218000400be00020040000a
:1092c800838048002e0190003001980041019800e9
:1092d8002e0090001e01be00120098002300980086
:1092e8002e00900030039000c003900086007800a4
:1092f800a0002000000ab8006030b900050178001d
:10930800000141006a38b90000014100820278007a
:109318000400be000080fa00000006000200fa0007
:10932800000f78001e007800beff07009e0078003e
:1093380010002000800878001e007800300390009c
:10934800c003900086007800a0002000000ab80042
:109358006030b90005017800000141006a38b900a1
:1093680000014100820278000400be000080fa007b
:10937800000006000200fa00000f78001e007800c6
:10938800a8ff07009e0078000000eb008008780026
:109398001e00780030039000c0039000860078001b
:1093a800a0002000000ab8006030b900050178006c
:1093b800000141006a38b9000001410082027800ca
:1093c8000400be000080fa00000006000600fa0053
:1093d80020079800240007000001be002e0090001e
:1093e80001002000001f4100019749001e000700ee
:1093f800be0f5000ae8f5800fcff39000080fa0005
:10940800000006000600fa00200798001600070072
:10941800008fbe002e009000e90f500008003600b3
:109428002e009000a2002000110009000280d80040
:10943800010020001e0f40005e974800040037001e
:1094480010002000010020001e0f40005e97480019
:1094580005000700be0f5000ae8f5800fcff390012
:109468000080fa00000006000000fa007c000700f7
:10947800d0518000e15180000080fa000000060011
:109488000000fa00f05180000080fa000000060099
:109498000800fa0020079800310798002e00900075
:1094a800be009000008fbe0000e1200001002000f7
:1094b800be0f1000ae8f18000300360000e1200038
:1094c80001002000008fbe001e00be00e00f50000b
:1094d800e08f580003003a0010002000010020002f
:1094e800008fbe009e007800400620000009b800ea
:1094f8001e0078006000b9000302780000024200f4
:109508009e009000400620000088b900000242003a
:1095180084017800028fbe00f0ff2f0001002000b8
:10952800be0f1000ae8f180003003600f0ff2f00aa
:1095380001002000008fbe001e0078002052880025
:109548000080fa00000006000800fa0020079800d2
:10955800310798002e009000be009000008fbe00da
:10956800803e200001002000be0f1000ae8f1800c2
:1095780003003600803e200001002000008fbe005e
:109588009000200001002000be0f1000ae8f1800d0
:1095980003003e00a000200001002000008fbe0054
:1095a8001e00be00a2002000030020007bef070081
:1095b800008fbe00f0ff2f0001002000be0f10003a
:1095c800ae8f180003003600f0ff2f0001002000c6
:1095d800008fbe001e007800305288000080fa001c
:1095e800000006000400fa0020528000010020005c
:1095f800008fbe001e00be004206200003002000af
:1096080066ef0700008fbe001e00be000080fa0053
:10961800000006000400fa0030528000010020001b
:10962800008fbe009e007800a0002000000ab8004d
:109638001e0078006000b9000501780000014100b3
:109648001e0090006a00b900000141008202780003
:10965800048fbe001e00be000080fa000000060055
:109668000200fa00c2518000d0518000e151800010
:10967800000f51001e0078006101b800d051800031
:10968800e15180000200400083804800d0518800ea
:10969800e15188000080fa0000000600809fbe00ab
:1096a8000000fa000000eb0030088800c05180007c
:1096b8000000e800c0518800105280000000e0005f
:1096c80004003200105280000000e90010528800a7
:1096d80016003700c2c2bf0001c8b30001406000d5
:1096e8000004e00004003a00005280000000e80096
:1096f80000528800020037000000eb00005288008a
:109708000152800030528000808f500007003600e0
:10971800f05180000000e800f05188000000eb00e4
:1097280000528800205280001052880084e0a9006e
:109738000080fa004f00be00004006000400fa0056
:10974800000f78001e007800100078000000e0008c
:1097580003003200e0ff2f00100798006f00370069
:109768001e007800c000900030009000e00f50000c
:10977800e08f5800080032001e0078003001900089
:10978800c001900000e1200001002000800f51007e
:10979800818f590003003600d0ff2f001007980072
:1097a8005e0037001e00780050019000e001900034
:1097b8009000200001002000800f5100818f590087
:1097c800080036001e00780050019000e00190006b
:1097d800803e200001002000800f5100818f590039
:1097e80003003600c0ff2f00100798004b00370019
:1097f8001e00780070019000800990000090200001
:10980800d1032000800f5100818f590003003600da
:10981800b0ff2f0010079800400037001e007800a6
:1098280010099000a009900000902000d1032000aa
:10983800800f5100818f590003003600a0ff2f00d0
:1098480010079800350037001e007800c008900007
:1098580030089000e00f5000e08f580008003200f8
:109868001e00780030099000c00990000090200088
:10987800d1032000800f5100818f5900030036006a
:1098880090ff2f0010079800240037001e00780072
:10989800e008900050089000e00f5000e08f58005a
:1098a800080032001e00780050099000e00990007e
:1098b800800c200001002000800f5100818f59008a
:1098c8000300360080ff2f001007980013003700b0
:1098d8001e0078008010900070089000e00f500083
:1098e800e08f5800080032001e00780070099000d0
:1098f8008011900000902000d1032000800f5100bb
:10990800818f59000300360070ff2f001007980060
:10991800020037000000eb00100798001e009000be
:109928000080fa00000006002a00fa0030179800ac
:109938000e80e80041022000c90007000e80e80000
:1099480021022000ad000700000f78000e80e8001b
:10995800101090009e0f5000030032000080eb00b2
:1099680040179800390037000e80e8009000780012
:109978003e109000010878000e80e80090009000ea
:109988003e109000110098000e80e800a0009000a2
:109998003e109000210098000e80e800c000900062
:1099a800300090003e11900030019800410198006d
:1099b8000e80e800e0009000500090003e119000fa
:1099c80050019800610198000e80e800800890001e
:1099d800700090003e1190007001980001099800f5
:1099e8000e80e800a0089000100890003e1190003a
:1099f80010099800210998000e80e800c00890001e
:109a0800300890003e1190003009980041099800f4
:109a18000e80e800e0089000500890003e11900089
:109a280050099800610998000e80e80080109000a5
:109a3800700890003e11900070099800011198007c
:109a48003e1090003dff0700401798004e10900010
:109a58000080fa00000006002800fa00201798008d
:109a68002e10900035ff07000000e00003003200d0
:109a78000080eb0030179800360037002e10900059
:109a880010007800000f78002e1090001000900051
:109a9800100798002e1090002000900020079800d2
:109aa8002e109000c0009000300090003007980001
:109ab800410798002e109000e000900050009000a0
:109ac80050079800610798002e10900080089000b9
:109ad8007000900070079800010f98002e109000f9
:109ae800a008900010089000100f9800210f98000f
:109af8002e109000c008900030089000300f980099
:109b0800410f98002e109000e00890005008900037
:109b1800500f9800610f98002e1090008010900050
:109b280070089000700f9800011798000e007800d8
:109b3800210220003100070010179800f1000700eb
:109b48000e00780041022000930007000000eb009f
:109b5800301798003e1090000080fa0000000600c0
:109b68002400fa00a0aa2a00000f78000000eb00e9
:109b7800100798000000eb00200798006000b8006c
:109b880030079800410798006000b8005007980017
:109b9800610798006000b80070079800010f9800ee
:109ba8006000b800100f9800210f98006000b800fe
:109bb800300f9800410f98006000b800500f9800cf
:109bc800610f98006000b800700f980001179800a6
:109bd8000e007800210220000800070010179800e6
:109be800c80007000e007800410220006a00070044
:109bf8000000eb000080fa00000006000800fa00f0
:109c080020079800310798000000eb00000f78004b
:109c18000000eb00100798000a0037001e009000b3
:109c2800800078002e0090000080400010407800ee
:109c38000000fb001e0f40001e0090000000e8001e
:109c4800100798009e0090003e009000808f500002
:109c5800f2ff35001e0078000080fa0000000600c0
:109c68001400fa0070079800010f98000e08900081
:109c78000000e000040034008e089000004020003e
:109c8800808f5000030034000080eb00100f980014
:109c98003e0037000e0890000000e9002200200076
:109ca800110009000200d8000000e8002007980011
:109cb8000000eb00000f78000000eb001007980090
:109cc8002c0037001e009000000040008000780043
:109cd8000000210000804000cf80de00300798009f
:109ce80041079800be0090004e009000ec0007006d
:109cf80050079800610798002e489000804078002f
:109d08007e009000014878007e0090000000e80086
:109d1800700798001e0fe8000e0890009e0f1000b4
:109d280003003a000000eb00100f980017003700fe
:109d38003e489000804078007e00900001487800fe
:109d48007e0090000000e800700798001e0fe800f1
:109d58000e0890009e0f100003003a000000eb0070
:109d6800100f9800090037001e0090000000e8005e
:109d7800100798009e0090002e009000808f5000e1
:109d8800d0ff35000000eb00100f98001e0890006f
:109d98000080fa00000006001400fa00700798001e
:109da800010f98000e0890000000e0000400340045
:109db8008e08900000402000808f5000030034007f
:109dc8000080eb00100f98004b0037000e08900041
:109dd8000000e90022002000110009000200d8005c
:109de8000000e800200798000000eb00000f780052
:109df8000000eb0010079800390037001e009000a3
:109e08000000400080007800000021000080400031
:109e1800cf80de0030079800410798001e0fe80049
:109e28000e0890000000e8009e0f100007003d009b
:109e38007e00900010407800204f98007e0090002f
:109e48000000e800700798000200370000c0eb002f
:109e5800204f98001e0fe8000e0890000000e80050
:109e68009e0f100007003d007e0090001040780013
:109e7800304f98007e0090000000e80070079800be
:109e88000200370000c0eb00304f98000040eb00a4
:109e9800404f98000040eb00504f98005e00900043
:109ea8006e019000be0090004e0290008001780084
:109eb800040078004e0007003b0007000e089000e1
:109ec8009e0f1000030035000000eb00100f9800f3
:109ed800090037001e0090000000e80010079800f5
:109ee8009e0090002e009000808f5000c3ff350028
:109ef8000000eb00100f98001e0890000080fa0088
:109f0800000006000400fa00000021000100200003
:109f1800008fbe009e0078001e00900043000700de
:109f28000080fa00000006000c00fa000000eb00b8
:109f3800100798000000eb00000f780014003700ad
:109f48001e00780000004000010020002007980053
:109f5800310798003e009000900188002e00900084
:109f68001000ba00400798002e0090001080ba0038
:109f7800500798004e009000de00900080007800a6
:109f88001e00900001004000100798001e0fe80016
:109f9800f0bf2a009e0f1000e9ff36001e00900057
:109fa8000080fa00000006000200fa0030002400d9
:109fb800003b88001e00780050052000303b8800d8
:109fc800a00a2000303b880061e7a80000000000dc
:109fd8000000000061c7bf0001c8b3000140600075
:109fe8000004e000fbff3a000080fa0000000600d1
:109ff8000800fa00000f780011079800220798005f
:10a00800330798001e007800900188009e00900099
:10a018003e0090008008bb009e0090002e0090003b
:10a028008088bb000080fa00000006000800fa00e3
:10a03800100798002107980090018000000f780011
:10a048001e0090009001880020042400003b880036
:10a05800ae0090002e0090008008bb003e009000eb
:10a0680050052000303b8800a00a2000303b8800c3
:10a0780061e7a800000000000000000061c7bf0001
:10a0880001c8b300014060000004e000fbff3a0093
:10a098001e007800900188000080fa000000060089
:10a0a8000800fa0020079800310798002e00900059
:10a0b800900188003e0090001000ba00000f780060
:10a0c8003e0090001080ba00100798001e00be00e5
:10a0d8000080fa00000006007400fa002c03a900b2
:10a0e8002c23a9002c43a8002c63a8002c83a800cb
:10a0f8002ca3a8002cc3a8002ce3a8002d03a800bb
:10a108002d23a8002d43a8002d63a8002d83a800a7
:10a11800616c20009140780000ceb30000c0600060
:10a128003040b300c6e6b700416a2000914078008d
:10a1380000ceb30000c060005040b300a4e6b700f2
:10a14800716c20009140780000ceb30000c0600020
:10a158005040b300c7e6b700616a2000914078001c
:10a1680000ceb30000c060000034a000a6e6b7002f
:10a17800516d20009140780000ceb30000c060000f
:10a188007040b300d5e6b700816a2000914078009e
:10a1980000ceb30000c060004041b300a8e6b7009d
:10a1a800316d20009140780000ceb30000c06000ff
:10a1b8000034a000d3e6b70061dd07003df80700d2
:10a1c8000604070031df0700ecfb0700df0007008b
:10a1d80077fa0700f1f40700e4004700c0962b0067
:10a1e800801f780050972b00801f780010982b0054
:10a1f800801f78000100780019e20700e687570001
:10a20800e40047001000200006de0700e4004700d5
:10a21800609a2b00801f7800b09b2b00801f78006d
:10a22800010078000ee20700e4875700e4004700c9
:10a2380010002000fbdd0700e09f2000bafd0700aa
:10a248000000e000270032000000eb00f04f88001b
:10a2580010002000005088001000200010508800d6
:10a268002000200001002000205088003150880084
:10a27800e001200001002000405088005150880073
:10a28800002f2d00010020006050880071508800c8
:10a2980080702000010020008050880091508800c4
:10a2a800c012200001002000a0508800b150880092
:10a2b8008007200001002000c0508800d15088008d
:10a2c800001e200001002000e0508800f1508800a6
:10a2d800c19c2b0010002000d2dd0700e09f200069
:10a2e800ddfd07000050800029f6070010508000af
:10a2f80051f60700205080003150800064fc0700b0
:10a3080040508000515080008ffc07006050800052
:10a318007150800094f507008050800091508000b3
:10a3280069f50700a0508000b150800062f6070070
:10a33800c0508000d1508000b3f50700e050800085
:10a34800f1508000e1f50700000037000080eb00c5
:10a358003cf50700640047002e0007000000e000fd
:10a3680003003a0030002000100798001000370062
:10a3780064004700a19f2b00d6010700000f78005a
:10a388001e007800104078000004e00003003a0046
:10a398002000200010079800050037004200200028
:10a3a800616d2b001e0078001f020700100798003f
:10a3b8001e009000e30f5000e4ff32001e009000e2
:10a3c8000000e0000f0032001e009000e20f500075
:10a3d8000c003200400520000e0040009e00900056
:10a3e800811f7800d19f2b00811f78009ce1070016
:10a3f800e4875700410520008e80400010002000af
:10a4080088dd070081a02b001000200085dd0700f3
:10a41800ceff37000800fa0030079800d0c0b3001c
:10a42800404798000000eb0010079800e50047003f
:10a438001000200022dd07000000e000400032008c
:10a44800de409000100020003edd07005e409000d6
:10a45800ed4f500003003a00a1c0b30010002000e7
:10a4680038dd0700de4090004e40900080cf50005d
:10a478001a0032005e409000e84f50000d00320094
:10a48800e14f8000f0042000808f500009003c005c
:10a49800e24f80005e40900080407800a097200046
:10a4a80000004100014878000200e800e04f880001
:10a4b80006003700e04f80000000e0000300340091
:10a4c800e04f80000000e900e04f8800be009000e7
:10a4d8000040eb0080487800190037001000200089
:10a4e80010079800e14f8000a0972000808040006e
:10a4f8000040eb00804878000000eb00000f780077
:10a508000a0037001e007800800078003e009000a6
:10a51800008140009e007800a09720000080400045
:10a5280010407800004978001e0fe800e04f8000d6
:10a538009e0f1000f3ff34000000eb00e04f88008e
:10a548001e0090000080fa00000006000000fa00db
:10a5580040002000d600070060002000d40007005b
:10a568001000200070de07001000200063de0700e6
:10a578000000eb0061de07000000eb006ade070068
:10a588001000200068de0700300020005bde0700b6
:10a598000000eb0059de07000000eb0057de070063
:10a5a8000000eb0055de07000d0037004052800028
:10a5b8005152800061004000e0804800405288000d
:10a5c800515288004252800053528000f0ff2f0001
:10a5d800f1002000800f5100818f590006003e00d5
:10a5e8000000eb0045de070080007800f00f200037
:10a5f800808f5000edff3a000000eb004ade0700b4
:10a608000080fa00000006000200fa004000200066
:10a61800a700070060002000a50007000006200032
:10a62800a300070001aa2b0010002000fddc070092
:10a63800a9000700000f780009003700a00f2000cc
:10a6480070fb0700a4000700000f7800c1aa2b00c8
:10a6580010002000f3dc07005000200079f4070008
:10a668009e007800618060000004e000f3ff3a007b
:10a67800e1aa2b0010002000eadc07006000b80007
:10a6880040528800515288000000eb000080fa0018
:10a69800000006000e00fa00881f780030079800b6
:10a6a800410798005207980063079800400020006f
:10a6b8007f00070088000700610060000004e000d8
:10a6c800fcff3a001000200017de070030002000d1
:10a6d8000ade07000e81e8003e009000ce009000e0
:10a6e8008a0007000e80e800204090000080fb00f0
:10a6f80002de07000e80e800104090000080fb009a
:10a70800fedd07000e80e800104078000080fb00a6
:10a71800fadd07000000eb00000f780008003700a2
:10a728001e007800800078005e00900000844000e1
:10a738000000eb00f1dd0700004c78001e0fe80078
:10a748006e0090009e0f1000f5ff35000000eb0032
:10a75800f5dd07000000eb004f0478000080fa00e8
:10a76800000006000800fa004047980042528000a6
:10a7780053528000f0ff2f00f1002000800f51009d
:10a78800818f5900030036000080eb0030079800e5
:10a79800270037004e4090000074a1004047980001
:10a7a8004d000700610060000004e000fcff3a0073
:10a7b800600020003e00070010002000dadd0700de
:10a7c80020002000cddd070040528000515280005b
:10a7d8000e0178004d0007002e4090000080fb001d
:10a7e800c6dd07001e4090000080fb00c3dd0700a7
:10a7f8001e4078000080fb00c0dd07004e4090003e
:10a808000000fb00bddd07000000eb00c6dd07000f
:10a81800405280005152800061004000e0804800b2
:10a8280040528800515288000000eb003007980021
:10a838003e0090000080fa00000006000600fa00c2
:10a84800100798000000eb00000f78000c0037009c
:10a858001e007800800078001e00900000804000f4
:10a86800104078001e0fe800beff07000000e0005f
:10a8780003003d000080eb00200798000900370026
:10a888001e007800800078001e00900000804000c4
:10a89800104078000004e000edff3a000000eb00f3
:10a8a800200798002e0090000080fa0000000600a3
:10a8b8000200fa00000f7800100020009add07005f
:10a8c8001e0078008ddd07000000eb0096dd070014
:10a8d8000080fa00000006000200fa0010002000c4
:10a8e80091dd07005000200084dd07000000eb0028
:10a8f80082dd0700000f78000000eb008add07000a
:10a908001e0078000080fa00000006000800fa0027
:10a918001007980021079800320798000000eb0004
:10a92800000f78000f0037001e00780080007800c4
:10a938003e009000808040001e0090008048780013
:10a948001e009000ae0090004809dd004800de00bf
:10a9580000007100c808de00100798002107980061
:10a968001e0fe800300020009e0f1000eeff34009c
:10a978000080fa00000006000800fa00881f78002e
:10a9880010079800210798000000eb00000f7800de
:10a998001e009000104078000004e00003003a0018
:10a9a8000000eb0030079800460037001e007800d2
:10a9b800800078002e009000008040001040780051
:10a9c8000000fb00e0e00700000478001e007800ab
:10a9d800800078001e009000008040001040780041
:10a9e8000000fb00d8e00700800f5400150032007b
:10a9f8002e0090000000e800200798002e0090002c
:10aa0800104078000004e00003003a000000eb006a
:10aa1800300798002b0037002e00900090407800f7
:10aa2800c0c7b30080cf5000f1ff3a002e0090005d
:10aa38000000e800200798000000eb00000f7800f5
:10aa48001b0037001e0fe8001e0078008000780009
:10aa58002e00900000804000104078000004e000c4
:10aa6800080032001e007800800078002e00900058
:10aa78000080400090407800c0c7b30080cf5000ed
:10aa88000b003a001e007800800078001e0090003d
:10aa98000080400010407800520007000000e000ed
:10aaa80003003a001e0078003007980005003700c0
:10aab800700220009e0f1000bcff34001e007800ba
:10aac800300798003e0090004f0478000080fa009c
:10aad800000006000600fa001007980021079800f9
:10aae8000080eb00000f78000e0037001e00900079
:10aaf800104178001e007800800078002e00900039
:10ab08000080400010407800804f510005003a0056
:10ab18001e0090000000e800100798000080eb007d
:10ab2800000f78001e0fe8001e00780080007800f3
:10ab38002e00900000804000104078000004e000e3
:10ab4800eaff3a001e0090000080fa0000000600ac
:10ab58000400fa00000f780021ac2b001e007800da
:10ab6800dcff0700000f78001e0078009040780096
:10ab7800d0c2b30080cf5000050032001e0078001c
:10ab880090407800b0c2b30080cf500001003a0076
:10ab98001e0fe80051ac2b001e007800cdff070007
:10aba800000f780071ac2b001e007800c9ff070069
:10abb800000f78001e007800104078000004e000c4
:10abc800030032000000eb00100798000200370075
:10abd80010002000100798001e0090000080fa0066
:10abe800000006000400fa00004f78001e00fb0079
:10abf8005ce007000000e00003003a00f0c5b30085
:10ac08009e4f100003003a00100020001007980023
:10ac1800020037000000eb00100798001e009000ab
:10ac28000080fa00000006000c00fa0020079800d7
:10ac380031079800420798000000eb00000f7800e9
:10ac480021ac2b002e009000a2ff070020079800df
:10ac58001e0037001e0078004200dd0080007800ea
:10ac68003e00900000804000900078002e00900088
:10ac780041ff0700100798001e0090000000e00048
:10ac8800110032001e009000800078002e00900015
:10ac98000080400021ac2b008eff070020079800a1
:10aca8001e0078004200dd00800078003e00900021
:10acb80000804000900090002e00900001000100ec
:10acc800500798000c0037001e0fe8001e0078009f
:10acd8004200dd00800078003e00900000804000c7
:10ace80010007800104078000004e000d9ff3a0016
:10acf8004e009000500798005e0090000080fa0017
:04ad08000000060041
:020000040000fa
:10ad0c00380a00000c00000000000000440a00009b
:10ad1c000400000002000000c80003000000000056
:10ad2c001809000062000000000000004c0a00003e
:10ad3c0002000000000000007a0900005000000032
:10ad4c0002000000000000000000000000000000f5
:10ad5c0000000000000000000000000000000000e7
:10ad6c0000000000000000000000000000000000d7
:10ad7c0000000000000000000000000000000000c7
:10ad8c0000000000000000000000000000000000b7
:10ad9c0000000000000000000000000000000000a7
:10adac000000000000000000000000000000000097
:10adbc00fc09000024000000000000004e0a000006
:10adcc000200000000000000000800001801000054
:10addc0000000000200a0000180000000200000023
:10adec0080f93700034077001b00010000e093005e
:10adfc000400010000c0d400010000005307000053
:10ae0c00ca0900003200000000000000500a0000d7
:10ae1c00020000000200000001000000480a0000cf
:10ae2c000400000000000000520a00004a0000006c
:10ae3c00020000000000210015110e000d0c0b008b
:10ae4c000b0a0a000909090009090800080808008a
:10ae5c00080808000707070007070700070707008f
:10ae6c00070707000730310032333400353637001e
:10ae7c0038396100626364006566670068696a005e
:10ae8c006b6c6d006e6f7000717273007475760070
:10ae9c00777879007a0000002e0b00001200000079
:10aeac000200000001000200000400000800100075
:10aebc0000000000202b2d00233000004c0b000064
:10aecc000800000002000000686a6c00747a4c00f4
:10aedc0000000000540b0000040000000200000001
:10aeec000000000000000000400b00000c000000ff
:10aefc0002000000686a6c00747a4c000063430026
:10af0c006e5b00000c0b0000220000000200000031
:10af1c003031320033343500363738003961620055
:10af2c00636465006600300031323300343536001e
:10af3c0037383900414243004445460000000000c8
:10af4c00e60a000026000000020000000a000800cb
:10af5c000a101000106469006f75780058700000ba
:10af6c003031320033343500363738003961620005
:10af7c00636465006641420043444500460000009e
:10af8c009c0a00004a000000020000000000410082
:10af9c0029211c0019171600151413001212110088
:10afac001111100010100f000f0f0f000e0e0e00dd
:10afbc000e0e0e000e0d0d000d0d0d000d3031009e
:10afcc00323334003536370038396100626364003f
:10afdc006566670068696a006b6c6d006e6f700067
:10afec007172730074757600777879007a000000be
:04affc000000000051
:020000040000fa
:10b000000600fa00004f7800110798001e0090001b
:10b01000440007000000e000030032000000eb00e5
:10b0200020079800100037001e0090009000780064
:10b030001e00900010009000008040001e48780024
:10b040001e009000100090008000e8001e0090009c
:10b0500030009000808060001e0090001100980079
:10b0600010002000200798002e0090000080fa00b9
:10b07000000006000600fa00000f78001107980093
:10b080001e0090003b0007000000e00006003200b8
:10b090009e0078000040eb00804878000000eb0044
:10b0a00020079800120037001e00900090007800e2
:10b0b0001e0090002000900000804000904078002a
:10b0c0001e007800014878001e00900020009000cb
:10b0d0008000e8001e00900030009000808060003a
:10b0e0001e0090002100980010002000200798000a
:10b0f0002e0090000080fa00000006000200fa0016
:10b10000000f78009e0078000000eb00a00098007f
:10b110009e0078000000eb00900098000080fa008c
:10b12000000006000400fa00000f78001e007800fe
:10b13000100090008000e8001e00780030009000b1
:10b14000808060001e00780020009000808f5000fa
:10b1500003003a001000200010079800020037009a
:10b160000000eb00100798001e0090000080fa001d
:10b17000000006000400fa00000f78001e007800ae
:10b18000a00090001e00780010009000808f5000fa
:10b1900003003a001000200010079800020037005a
:10b1a0000000eb00100798001e0090000080fa00dd
:10b1b000000006000200fa00000f78001e00780070
:10b1c000900090001e0078002000900080805000c9
:10b1d0001e00780030009000008060000080fa00bf
:04b1e0000000060065
:020000040000fa
:101e94000000fa002c83a8002ca3a8002d03a8009e
:101ea400d442a80000000000d042a90000000000b5
:101eb400c482a80000000000c082a9000000000045
:101ec40042c2a8004302a9004322a90042a2a800da
:101ed40042c2bf003040b30042e2b70021242000d8
:101ee4009140780030ceb30000c060008041b30060
:101ef40042e2b70041e2a8000080fa0000000600b8
:101f04000200fa00000f78001e00780040128800da
:101f140040c2bf00614060000004e000fcff3200ea
:101f2400401280000080fa00000006000200fa005f
:101f3400000f78001e00e00002003200d442a90025
:101f440001003700d442a800000000000080fa001d
:101f5400000006000200fa00000f78001e00e000f6
:101f640002003200c482a90001003700c482a80024
:0c1f7400000000000080fa0000000600e1
:020000040000fa
:10b1e4000000fa002ca3a9002c83a900000e200063
:10b1f400001988000000eb001019880020f02000de
:10b20400201988000000eb008019880021e3a800c1
:10b214000080fa00000006000600fa0010079800fb
:10b224001e009000200798002e009000e40f5000ac
:10b23400040032002e009000e50f5000040032009c
:10b244000600370040002000401988000500370040
:10b2540050002000401988000200370050002000f0
:10b26400401988002023a80020c3bf00624060006a
:10b274000004e000fcff3a0020c3bf00614060000e
:10b284000004e000fcff320000188000000f78008a
:0cb294001e0078000080fa000000060098
:020000040000fa
:101f80000000fa00705280000000e00001003a00fa
:101f9000ff3ffc00705280000000e8007052880093
:101fa0000080fa00000006000000fa007052800075
:101fb0000000e90070528800705280000000e000cc
:101fc00001003a000000fc000080fa00000006005a
:020000040000fa
:041fd0000000fe000f
:00000001FF
